S00F0000746563776172652E737265632A
S3150800280000C0002065CA0008C5520008D352000857
S31508002810E1520008EF520008FD52000800000000CF
S3150800282000000000000000000000000051C500087C
S315080028300B53000800000000F1C500080D530008FE
S31508002840B5CA0008B5CA0008B5CA0008B5CA00085E
S31508002850B5CA0008B5CA0008B5CA0008B5CA00084E
S31508002860B5CA0008B5CA0008B5CA0008B5CA00083E
S315080028702553000835530008B5CA0008B5CA00082C
S31508002880B5CA0008B5CA00084553000855530008DC
S31508002890655300087553000885530008B5CA000833
S315080028A0B5CA0008B5CA0008B5CA0008B5CA0008FE
S315080028B0B5CA00080000000000000000B5CA0008FC
S315080028C0B5CA000800000000000000009553000883
S315080028D000000000B5CA0008B5CA000800000000DC
S315080028E0B5CA0008B5CA00080000000000000000CC
S315080028F000000000000000000000000000000000CA
S31508002900000000000000000000000000B5CA000832
S315080029100000000000000000B5CA0008B5CA00089B
S31508002920B5CA0008B5CA0008A5530008B5CA000804
S31508002930B5CA000800000000000000000000000002
S31508002940B5CA0008B5CA0008B5CA0008B5CA00085D
S31508002950B5CA0008B5CA0008B5CA0008B5CA00084D
S31508002960B5CA0008B5CA0008B5CA000800000000C4
S31508002970B5CA0008B5CA000800000000000000003B
S31508002980B5CA0008B5CA0008B5CA00082255AAEE95
S3150800299010B5054C237833B9044B13B10448AFF38B
S315080029A000800123237010BD1801002000000000DC
S315080029B098CC000808B5034B1BB103490348AFF38D
S315080029C0008008BD000000001C01002098CC00080B
S315080029D081F0004102E000BF83F0004330B54FEAC2
S315080029E041044FEA430594EA050F08BF90EA020F2F
S315080029F01FBF54EA000C55EA020C7FEA645C7FEAC2
S31508002A00655C00F0E2804FEA5454D4EB5555B8BFE4
S31508002A106D420CDD2C4480EA020281EA030382EA55
S31508002A20000083EA010180EA020281EA0303362DE7
S31508002A3088BF30BD11F0004F4FEA01314FF4801CBA
S31508002A404CEA113102D0404261EB410113F0004FCC
S31508002A504FEA03334CEA133302D0524263EB430383
S31508002A6094EA050F00F0A780A4F10104D5F1200E21
S31508002A700DDB02FA0EFC22FA05F2801841F100017C
S31508002A8003FA0EF2801843FA05F359410EE0A5F150
S31508002A9020050EF1200E012A03FA0EFC28BF4CF081
S31508002AA0020C43FA05F3C01851EBE37101F0004537
S31508002AB007D54FF0000EDCF1000C7EEB00006EEB44
S31508002AC00101B1F5801F1BD3B1F5001F0CD34908CE
S31508002AD05FEA30004FEA3C0C04F101044FEA445225
S31508002AE012F5800F80F09A80BCF1004F08BF5FEAAC
S31508002AF0500C50F1000041EB045141EA050130BD8C
S31508002B005FEA4C0C404141EB0101013C28BFB1F59D
S31508002B10801FE9D291F0000F04BF01460020B1FAE8
S31508002B2081F308BF2033A3F10B03B3F120020CDABB
S31508002B300C3208DD02F1140CC2F10C0201FA0CF099
S31508002B4021FA02F10CE002F11402D8BFC2F1200CFE
S31508002B5001FA02F120FA0CFCDCBF41EA0C019040B4
S31508002B60E41AA2BF01EB0451294330BD6FEA0404FD
S31508002B701F3C1CDA0C340EDC04F11404C4F12002E8
S31508002B8020FA04F001FA02F340EA030021FA04F3FA
S31508002B9045EA030130BDC4F10C04C4F1200220FA51
S31508002BA002F001FA04F340EA0300294630BD21FA8F
S31508002BB004F0294630BD94F0000F83F4801306BF55
S31508002BC081F480110134013D4EE77FEA645C18BF49
S31508002BD07FEA655C29D094EA050F08BF90EA020FE0
S31508002BE005D054EA000C04BF1946104630BD91EAD8
S31508002BF0030F1EBF0021002030BD5FEA545C05D1DB
S31508002C004000494128BF41F0004130BD14F5800419
S31508002C103CBF01F5801130BD01F0004545F0FE418D
S31508002C2041F470014FF0000030BD7FEA645C1ABFC2
S31508002C30194610467FEA655C1CBF0B46024650EAF9
S31508002C40013406BF52EA033591EA030F41F4002125
S31508002C5030BD00BF90F0000F04BF0021704730B5AB
S31508002C604FF4806404F132044FF000054FF0000180
S31508002C7050E700BF90F0000F04BF0021704730B541
S31508002C804FF4806404F1320410F0004548BF404216
S31508002C904FF000013EE700BF42004FEAE2014FEA6B
S31508002CA031014FEA02701FBF12F07F4393F07F4F46
S31508002CB081F06051704732F07F4208BF704793F049
S31508002CC07F4F04BF41F40021704730B54FF460745C
S31508002CD001F0004521F000411CE700BF50EA01025F
S31508002CE008BF704730B54FF000050AE050EA010208
S31508002CF008BF704730B511F0004502D5404261EB78
S31508002D0041014FF4806404F132045FEA915C3FF4B8
S31508002D10D8AE4FF003025FEADC0C18BF03325FEA55
S31508002D20DC0C18BF033202EBDC02C2F1200300FA06
S31508002D3003FC20FA02F001FA03FE40EA0E0021FA2B
S31508002D4002F11444BDE600BF70B54FF0FF0C4CF419
S31508002D50E06C1CEA11541DBF1CEA135594EA0C0FCB
S31508002D6095EA0C0F00F0DEF82C4481EA030621EA06
S31508002D704C5123EA4C5350EA013518BF52EA033541
S31508002D8041F4801143F4801338D0A0FB02CE4FF0F3
S31508002D900005E1FB02E506F00042E0FB03E54FF023
S31508002DA00006E1FB03569CF0000F18BF4EF0010E1B
S31508002DB0A4F1FF04B6F5007F64F5407404D25FEA17
S31508002DC04E0E6D4146EB060642EAC62141EA5551CA
S31508002DD04FEAC52040EA5E504FEACE2EB4F1FD0C0C
S31508002DE088BFBCF5E06F1ED8BEF1004F08BF5FEA8A
S31508002DF0500E50F1000041EB045170BD06F000463C
S31508002E0046EA010140EA020081EA0301B4EB5C04E8
S31508002E10C2BFD4EB0C0541EA045170BD41F48011E0
S31508002E204FF0000E013C00F3AB8014F1360FDEBF05
S31508002E30002001F0004170BDC4F10004203C35DAE1
S31508002E400C341BDC04F11404C4F1200500FA05F364
S31508002E5020FA04F001FA05F240EA020001F0004205
S31508002E6021F0004110EBD37021FA04F642EB06017B
S31508002E705EEA430E08BF20EAD37070BDC4F10C04A5
S31508002E80C4F1200500FA04F320FA05F001FA04F269
S31508002E9040EA020001F0004110EBD37041F1000155
S31508002EA05EEA430E08BF20EAD37070BDC4F1200560
S31508002EB000FA05F24EEA020E20FA04F301FA05F2C8
S31508002EC043EA020321FA04F001F0004121FA04F270
S31508002ED020EA020000EBD3705EEA430E08BF20EA40
S31508002EE0D37070BD94F0000F0FD101F0004640007A
S31508002EF041EB010111F4801F08BF013CF7D041EAFC
S31508002F00060195F0000F18BF704703F000465200FF
S31508002F1043EB030313F4801F08BF013DF7D043EAD0
S31508002F200603704794EA0C0F0CEA135518BF95EA86
S31508002F300C0F0CD050EA410618BF52EA4306D1D10D
S31508002F4081EA030101F000414FF0000070BD50EA2C
S31508002F50410606BF1046194652EA430619D094EAB6
S31508002F600C0F02D150EA013613D195EA0C0F05D1A0
S31508002F7052EA03361CBF104619460AD181EA0301F4
S31508002F8001F0004141F0FE4141F470014FF00000AC
S31508002F9070BD41F0FE4141F4780170BD70B54FF047
S31508002FA0FF0C4CF4E06C1CEA11541DBF1CEA1355C7
S31508002FB094EA0C0F95EA0C0F00F0A7F8A4EB0504A9
S31508002FC081EA030E52EA03354FEA013100F08880A0
S31508002FD04FEA03334FF0805545EA131343EA126369
S31508002FE04FEA022245EA111545EA10654FEA00261E
S31508002FF00EF000419D4208BF964244F1FD0404F5D7
S31508003000407402D25B084FEA3202B61A65EB030532
S315080030105B084FEA32024FF480104FF4002CB6EBEF
S31508003020020E75EB030E22BFB61A754640EA0C006F
S315080030305B084FEA3202B6EB020E75EB030E22BFAF
S31508003040B61A754640EA5C005B084FEA3202B6EBF0
S31508003050020E75EB030E22BFB61A754640EA9C00AF
S315080030605B084FEA3202B6EB020E75EB030E22BF7F
S31508003070B61A754640EADC0055EA060E18D04FEA3D
S31508003080051545EA16754FEA06164FEAC30343EADD
S3150800309052734FEAC2025FEA1C1CC0D111F4801FAA
S315080030A00BD141EA00014FF000004FF0004CB6E7A3
S315080030B011F4801F04BF01430020B4F1FD0C88BF42
S315080030C0BCF5E06F3FF6AFAEB5EB030C04BFB6EB4D
S315080030D0020C5FEA500C50F1000041EB045170BD40
S315080030E00EF0004E4EEA113114EB5C04C2BFD4EB6D
S315080030F00C0541EA045170BD41F480114FF0000EF1
S31508003100013C90E645EA060E8DE60CEA135594EA6C
S315080031100C0F08BF95EA0C0F3FF43BAF94EA0C0F6F
S315080031200AD150EA01347FF434AF95EA0C0F7FF4E4
S3150800313025AF104619462CE795EA0C0F06D152EA38
S3150800314003353FF4FDAE1046194622E750EA41061C
S3150800315018BF52EA43067FF4C5AE50EA41047FF42D
S315080031600DAF52EA43057FF4EBAE12E74FF0FF3C92
S3150800317006E000BF4FF0010C02E000BF4FF0010C63
S315080031804DF804CD4FEA410C7FEA6C5C4FEA430CDC
S3150800319018BF7FEA6C5C1BD001B050EA410C0CBF2B
S315080031A052EA430C91EA030F02BF90EA020F00208D
S315080031B0704710F1000F91EA030F58BF994208BFF4
S315080031C090422CBFD8176FEAE37040F001007047B1
S315080031D04FEA410C7FEA6C5C02D150EA013C07D108
S315080031E04FEA430C7FEA6C5CD6D152EA033CD3D053
S315080031F05DF8040B704700BF8446104662468C464D
S315080032001946634600E000BF01B5FFF7B7FF00287F
S3150800321048BF10F1000F01BD4DF808EDFFF7F4FFA8
S315080032200CBF012000205DF808FB00BF4DF808ED33
S31508003230FFF7EAFF34BF012000205DF808FB00BF56
S315080032404DF808EDFFF7E0FF94BF012000205DF878
S3150800325008FB00BF4DF808EDFFF7CEFF94BF01202D
S3150800326000205DF808FB00BF4DF808EDFFF7C4FF26
S3150800327034BF012000205DF808FB00BF4FEA410279
S31508003280B2F1E04324BFB3F5001CDCF1FE5C0DD9B6
S3150800329001F0004C4FEAC0024CEA5070B2F1004F00
S315080032A040EB830008BF20F00100704711F0804F03
S315080032B021D113F13872BCBF01F00040704741F4C8
S315080032C080114FEA5252C2F11802C2F1200C10FACC
S315080032D00CF320FA02F018BF40F001004FEAC123B0
S315080032E04FEAD32303FA0CFC40EA0C0023FA02F354
S315080032F04FEA4303CCE77FEA625307D150EA01332A
S315080033001EBF4FF0FE4040F44000704701F00040F9
S3150800331040F0FE4040F40000704700BF08B52D4B52
S31508003320D3F8945001F060F900F0010401F04EFB67
S31508003330044000F02FFC044015F0005F3CD115F066
S31508003340805F3DD101F0BAF8044000F097FE0440D2
S3150800335000F0F0FE044001F065F9044000F0CEFCF0
S31508003360044001F0DDFA044000F0E2FF044000F0FA
S31508003370C3F9044000F01CF9044225D106F05AFDB1
S31508003380002000F08FF9022001F022F9124B1B6889
S315080033909B0B642202FB03F3002BF4D000BF00BF93
S315080033A000BF00BF00BF00BF00BF00BF00BF00BF17
S315080033B000BF00BF013BEFE7084801F01DF9C1E770
S315080033C0074801F019F9BDE7064B186806F0A1FD94
S315080033D0FEE700BF0010024094000020010000092B
S315080033E0020000093401002008B5054A00210548F5
S315080033F006F035FD044B1860003818BF012008BDDB
S315080034001CCE00081D3300083401002000B585B025
S31508003410EC468CE80F0000231A466146054800680A
S3150800342006F097FF0121044B186806F01FFE05B049
S315080034305DF804FB440100204001002008B5014660
S31508003440024B186806F012FE08BD00BF40010020B6
S3150800345030B589B08BE000231A4602A94E480068A9
S3150800346006F0B9FF9DF808509DF81130012B12D0CF
S31508003470022B35D0002B40F08780082D3CD86AB245
S31508003480002A69D0013D072D66D8DFE805F03D41E1
S3150800349045654C4F5B62142D0DD9404801F0ACF8D8
S315080034A0FF238DF818309DF81130059A012106A8DA
S315080034B000F08CFF68E0284600F038FB01908DF894
S315080034C0185004220DF119010DEB020001F094FFCA
S315080034D09DF81130059A052106A800F077FF53E0FC
S315080034E004220DEB02010DF1090001F085FF019997
S315080034F0284600F0ABFA47E0FF2D2DD1002000F05A
S31508003500D1F803F025FA3FE0012000F0CBF83BE0C4
S31508003510002000F0C7F837E040F6B831204B1868AD
S3150800352006F068FD30E001F061F82DE006228DF81E
S3150800353018200B228DF81920059A022106A800F0FA
S3150800354045FF21E000F038FBF0B9164801F054F8C1
S315080035501AE000F051FB17E0134801F04DF813E0AC
S31508003560022001F035F812E0002000F09BF84FF039
S31508003570FF33002207210D48006806F0C4FD044603
S3150800358010F0010F7FF467AF14F0020FE8D114F0C2
S31508003590040FECD0E8E700BF440100200100000852
S315080035A0380100200400000802000008400100203D
S315080035B070B52A4806F038FD294B1860041E18BF56
S315080035C00124284A0021284806F049FC274B1860A0
S315080035D000280CBF002404F00104254A1021082005
S315080035E006F06CFE234B186000280CBF002404F07C
S315080035F00104214D214B02220121284606F0A6FC92
S315080036001F4E306000280CBF002404F001041D4B37
S3150800361004220121284606F099FC1B4D2860002843
S315080036200CBF002404F001044FF47A71306806F0E8
S31508003630E1FC002814BF002404F0010440F6B83168
S31508003640286806F0D7FC002814BF002404F00104FB
S315080036500E4800F0E3FE204670BD00BF60CE0008AD
S315080036604001002088CE0008513400084801002097
S3150800367070CE0008440100203D34000850CE0008F2
S315080036803C01002040CE0008380100200D34000817
S3150800369008B50146024B186806F0E8FC08BD00BFED
S315080036A04C01002010B504460146032000F054FFE3
S315080036B02146122000F02CFA10BD08B5122000F0A1
S315080036C049FA08BD08B5F2EE087AB4EEE70AF1EE53
S315080036D010FA09DCF9EE047AB4EEE70AF1EE10FA0C
S315080036E004D5B9EE040A01E0B2EE080A00F06AFD54
S315080036F000F0010008BD000038B5174A0021174838
S3150800370006F0ADFB164B1860041E18BF01241548B9
S3150800371006F08AFC144B186000280CBF002404F03D
S315080037200104124B01221146114806F00FFC114DF7
S31508003730286000280CBF002404F001049FED0E0A3F
S31508003740FFF7C0FFC821286806F054FC002814BFFC
S31508003750002004F0010038BDCCCE00087D370008F3
S3150800376054010020ACCE00084C010020BCCE000855
S3150800377091360008500100200000000008B52DED24
S315080037800C8BDFED759AB0EE699AF0EE698AB0EEA9
S31508003790698A45E00020FFF785FF704800F02CFF96
S315080037A06FE09FED6D9AF4EEE7CAF1EE10FA02D5D6
S315080037B07CEEE76A01E0DFED686AB4EEC79AF1EEDF
S315080037C010FA07D4F4EEC76AF1EE10FA00F3958002
S315080037D0B0EE479A3DEE0D7A78EEEAAA27EE2A7AF7
S315080037E0DFED5F6A6BEEA66A37EE267AF1EE479A48
S315080037F079EE277A77EEC77AF4EECC7AF1EE10FAFC
S3150800380006DCF4EEEC7AF1EE10FA79D4B0EE67CA7B
S31508003810B0EE4C0AFFF756FF10B9524800F0ECFE1E
S31508003820F0EE69BAB0EE49BAF0EE68AAB0EE48AA68
S315080038304FF0FF33002201214B48006806F063FC75
S3150800384010F0010FF4D0494803F089FFFFF735FF60
S315080038509FED418AF0EE488AB0EE489AF0EE489A13
S315080038600028DDD0002000F075F900284BD10E2085
S3150800387000F074F9DFED3E7AB4EEE70AF1EE10FADD
S3150800388088DC022000F06AF9B0EE409A032000F0C6
S3150800389065F9F0EE409A042000F060F9B0EE40DADF
S315080038A0062000F05BF9B0EE40CA072000F056F992
S315080038B0F0EE40CA092000F051F9F0EE408A0520E2
S315080038C000F04CF938EEC08A69EE087AB6EE007A4E
S315080038D029EE877ADFED276A27EE267A3AEE08AAD6
S315080038E027EE0A7A37EE0B7AB4EEE7CAF1EE10FA4B
S315080038F07FF757AF3CEE679A55E7B0EE669A69E7E9
S31508003900B0EE6CCA84E7002000F024F9012808D03C
S31508003910F0EE6B9AB0EE4B9AF0EE6A8AB0EE4A8AEF
S315080039207EE700F01BF9FFF7CDFE40B1DFED0A9AFE
S31508003930B0EE699AF0EE698AB0EE698A70E70E48C9
S3150800394000F05AFEDFED049AB0EE699AF0EE698A45
S31508003950B0EE698A64E700BF0000000004000007B3
S315080039609A99193F020000074C01002064030020C1
S315080039700000DC42CDCC4C3E0100000701288CBF7C
S315080039800020012070470000084B03EB00139B68DA
S315080039908B4207D8054B03EB0013DB688B4203D237
S315080039A000207047002070470120704700CF0008AC
S315080039B0084B03EB00139B688B4207DC054B03EBB4
S315080039C00013DB688B4203DA00207047002070473B
S315080039D00120704700CF00080C4B03EB0013D3ED12
S315080039E0027AF4EEC07AF1EE10FA0BD8074B03EB25
S315080039F00013D3ED037AF4EEC07AF1EE10FA03DA87
S31508003A0000207047002070470120704700CF00084B
S31508003A1008B503010C4AD35C13F0010F09D113F062
S31508003A20020F0BD113F0040F0BD00846FFF7A6FFC1
S31508003A3003E000EE101AFFF7CFFF08BDFFF7B8FF47
S31508003A40FBE7FFF7A1FFF8E700CF000838B5044603
S31508003A500301144AD35C13F0080F13D10D464FF037
S31508003A60FF31114B186806F0D3FB29462046FFF7AD
S31508003A70CFFF78B10D4B43F834500B4B186806F05E
S31508003A80F6FB38BD000240F0C06040F0040000F0CC
S31508003A90B3FDF6E7200240F0C06040F0080000F0F1
S31508003AA0ABFDEAE700CF0008580100205C010020C2
S31508003AB038B504460D464FF0FF31134B186806F02B
S31508003AC0A7FB082C0CD029462046FFF7A1FF60B1BA
S31508003AD00E4B43F834500C4B186806F0C8FB38BD3B
S31508003AE000F06EFC0828F3D1EDE7084B03EBC4039E
S31508003AF01A7942F002021A71200240F0C06040F0C2
S31508003B00100000F079FDE3E7580100205C01002071
S31508003B1008B5FFF7CDFF08BD00B583B08DED010AE6
S31508003B200199FFF7C5FF03B05DF804FB38B50446F5
S31508003B30064D4FF0FF31286806F06AFB044B53F830
S31508003B403440286806F093FB204638BD580100200B
S31508003B505C01002008B5FFF7E9FF08BD08B5FFF7C7
S31508003B60E5FF00EE100A08BD08B5034B03EB00138A
S31508003B705968FFF79DFF08BD00CF000810B500245F
S31508003B8004E0E0B2FFF7F0FF0134A4B2142CF8D930
S31508003B9010BD000010B5064806F0EFFA054B186090
S31508003BA0041E18BF0124FFF7E9FF204610BD00BF19
S31508003BB0F0CE00085801002038B500F0F7FE00F0F6
S31508003BC00105002401E00134E4B2142C0ED82301C7
S31508003BD0084AD35C13F0100FF5D02046FFF7A6FF6E
S31508003BE00146204600F0B5FE0540ECE700F0D0FEA1
S31508003BF0284038BD00CF000830B583B00024012521
S31508003C0001E00134E4B2142C10D82301124AD35C23
S31508003C1013F0100FF5D001A9204600F093FE0540D9
S31508003C20EFD001992046FFF743FFEAE70DB103B04D
S31508003C3030BD0A4800F0E0FC002401E00134E4B29B
S31508003C40142CF4D82301044AD35C13F0100FF5D0D2
S31508003C502046FFF789FFF1E700CF0008200000069D
S31508003C6008B572B10D4B60F07F00187000225A70CB
S31508003C7099700B480323838100F0E2FC00F00100F1
S31508003C8008BD064B60F07F0018705970044802237F
S31508003C90838100F0D5FC00F00100F1E7080200205E
S31508003CA00000002010B50C4692B1114B1870002286
S31508003CB05A709A700F480323838100F0C1FC00F004
S31508003CC001000D4B5A789B7843EA0223238010BDE6
S31508003CD0074B187000225A7006480223838100F0A9
S31508003CE0AFFC00F00100044B5B782380EFE700BFD0
S31508003CF008020020000000201002002038B51448F1
S31508003D0006F03BFA134D2860041E18BF01244FF035
S31508003D10FF3106F07DFA002000F0B0FB0022822178
S31508003D201046FFF79DFF0440002000F0B7FB012076
S31508003D3000F0A4FB002282211046FFF791FF044001
S31508003D40012000F0ABFB286806F091FA204638BD42
S31508003D5050D00008040200202DE9F04182B00F4639
S31508003D60904600230B70ADF8063018B1012854D0E0
S31508003D70012600E00126404D4FF0FF31286806F085
S31508003D8047FA304600F07AFB0022A0211046FFF7DA
S31508003D9067FF00F00104304600F080FB286806F053
S31508003DA066FA642006F0C4F84FF0FF31286806F07A
S31508003DB02FFA304600F062FB01220DF1060110468B
S31508003DC0FFF770FF0440304600F068FB286806F0ED
S31508003DD04EFA24B3BDF8063013F0010F24D15B0860
S31508003DE0ADF80630A8F80030234D4FF0FF312868AB
S31508003DF006F00EFA304600F041FB002284211046F8
S31508003E00FFF72EFF0440304600F048FB286806F00E
S31508003E102EFA204602B0BDE8F0810026ABE73B78D3
S31508003E2043F002033B70F4E7134C4FF0FF31206870
S31508003E3006F0EEF9304600F021FB0022394607204D
S31508003E40FFF730FF304600F029FB304600F016FB3E
S31508003E50002282211046FFF703FF304600F01EFBC2
S31508003E60206806F004FA3B7803F0FC033B7043F045
S31508003E7001033B700024CCE7040200200000000088
S31508003E80F0B585B0012006F053F80822704971484C
S31508003E9002F022F8B9E004244FF0FF316E4B18689F
S31508003EA006F0B6F900230AE0E118694A32F811105B
S31508003EB004AA02EB830242F8101C01339BB2032BBF
S31508003EC0F2D91420FFF74AFE002325E004AA02EBE4
S31508003ED0830252ED047AF8EE677A9FED607A67EE10
S31508003EE0877A9FED5F7A67EE877A67EE807A5D4A12
S31508003EF002EB830292ED007A67EE277A5A4A02EBC2
S31508003F00830292ED007A77EEC77A584A02EB83026B
S31508003F10C2ED007A01339BB2032BD7D9002401E006
S31508003F200134A4B2032C1DD8504B03EB8403186844
S31508003F30FEF7B2FE06460F4641A3D3E90023FFF774
S31508003F4089F90028ECD040A3D3E900233046394646
S31508003F50FFF76CF90028E3D0444B03EB84030022F7
S31508003F601A60DDE7002301E001339BB2032B14D866
S31508003F703F4A52F82320002AF6D13C4A02EB830234
S31508003F80D2ED007AF5EEC07AF1EE10FAECD5374AA2
S31508003F9002EB830200211160E6E7344C94ED020A35
S31508003FA00B20FFF7B9FD94ED030A0C20FFF7B4FDCB
S31508003FB0D4ED037AF5EE407AF1EE10FA36D19FED9C
S31508003FC02D0A0D20FFF7A8FD284C94ED020AD4ED22
S31508003FD0037A20EE270A0E20FFF79EFD94ED000ACD
S31508003FE00F20FFF799FD94ED010A1020FFF794FDC5
S31508003FF094ED000AD4ED017A20EE270A1120FFF786
S315080040008BFD154B186806F032F94FF0FF33002286
S3150800401003211948006806F076F810F0020F7FF4BD
S315080040203AAF10F0010FF0D0002435E70F4B93EDAF
S31508004030020A80EE270A0D20FFF76EFDC4E700BFCF
S315080040409A9999999999B9BF9A9999999999B93FC4
S315080040503402002070040020280200200000803D61
S3150800406000008039C4D00008B4D000081802002027
S31508004070A4D00008000000002C02002010B50F4A4A
S3150800408000210F4805F0EBFE0E4B1860041E18BF02
S3150800409001240D4805F0C8FF0C4B186000280CBF1A
S315080040A0002404F001040A4806F067F8094B186072
S315080040B000280CBF002004F0010010BD80D00008C5
S315080040C0813E00083002002070D000082C02002033
S315080040D060D000082802002008B50221024B1868A3
S315080040E005F0C4FF08BD00BF2C02002008B5012159
S315080040F0024B186805F0BAFF08BD00BF2C02002065
S3150800410008B5836D33B9C36CD86B40F0806000F096
S3150800411073FA08BD806D40F0407000F06DFAF8E75C
S3150800412008B50146024B186805F0A0FF08BD00BF98
S315080041304C02002038B51A4A00211A4805F08FFEAD
S31508004140194B1860041E18BF0124184805F06CFFA7
S31508004150174B186000280CBF002404F00104154B07
S3150800416001221146144805F0F1FE144D2860002876
S315080041700CBF002404F001040021114802F08EFC53
S31508004180002814BF002404F001043221286805F031
S3150800419031FF002814BF002004F0010038BD00BF1D
S315080041A0F4D000080D43000854020020D4D00008BB
S315080041B04C020020E4D000082141000850020020EB
S315080041C0C803002008B5064B83ED000A0121054BFC
S315080041D0186805F04BFFB0FA80F0400908BD00BF2B
S315080041E0440200204C02002008B52DED028B10EE8B
S315080041F0100AFEF751FD11A3D3E90023FEF7EEFBE3
S3150800420010A3D3E90023FEF7C9FEFFF737F808EE37
S31508004210100ADFED097A28EE278A1420FFF79EFC9C
S31508004220C8EE007AFCEEE77A17EE900ABDEC028B30
S3150800423008BD00BFAFF3008000F07F454A0C022B93
S3150800424087163440166BB8C83D0D41400000000083
S3150800425008B52DED028B2A4BD3ED007A294B93ED49
S31508004260008AF4EEC87AF1EE10FA26D517EE900A0F
S31508004270FEF712FD20A3D3E90023FEF7AFFBFEF7F6
S31508004280FDFF07EE900A1E4B1860B4EEE78AF1EEC2
S3150800429010FA01D583ED008A194B93ED000AFFF752
S315080042A0A3FF034600221146174802F029FCB0FA7C
S315080042B080F04009BDEC028B08BDF4EEC87AF1EE39
S315080042C010FAE9DD17EE900AFEF7E6FC0AA3D3E931
S315080042D00023FEF781FBFEF7D1FF07EE900A084B95
S315080042E01860B4EEE78AF1EE10FAD5DD83ED008AA0
S315080042F0D2E700BFAFF300809A9999999999B93F87
S315080043004802002044020020C803002008B54FF0E8
S31508004310FF33002201210548006805F0F4FE10F07D
S31508004320010FF4D0FFF794FFF1E700BF4C0200201D
S3150800433070B5042000F02CF91D4C23780343237034
S31508004340032000F025F9237843EA4003237002206E
S3150800435000F01EF9237843EA80032370012000F059
S3150800436017F9237843EAC000C0B22070114E3368AB
S3150800437043EA40133360104D1049284601F04DFFBB
S3150800438004463146284601F048FF0443E4B228466D
S3150800439001F0C6FF0443E4B20221284602F018F9E8
S315080043A0204310F0FF0F0CBF0120002070BD00BF96
S315080043B05802002044000020000400206C00002061
S315080043C0014B1878704700BF58020020082901D908
S315080043D00020704700B587B012021FFA82FC4CEA2B
S315080043E003130C4A1278134343F410730093002303
S315080043F001930293039304918DF814300123024626
S315080044006946054801F0BAFFB0FA80F0400907B0DE
S315080044105DF804FB5802002000040020014B1860D8
S31508004420704700BF5C02002030B58FB005AB07AA05
S31508004430002102F018F8079BC3F300220492C3F385
S3150800444001138DF80D309DF82C208DF80C2001AC49
S31508004450214605A800F0D0FF034B1D6894E80F001D
S31508004460A8470FB030BD00BF5C02002008B5406AFF
S3150800447040F0807000F0C0F808BD000008B5064B93
S315080044804FEA401C03EB4010027F818853F80C006A
S3150800449003F063F808BD00BF18D1000808B5064B3D
S315080044A04FEA401C03EB4010027E818853F80C004B
S315080044B003F053F808BD00BF18D1000870B582B0E4
S315080044C0224B1A6E42F001021A661B6E03F00103B4
S315080044D00193019B012500240BE000231D401C4B82
S315080044E04A0103EB41110431985802F057FF013491
S315080044F0E4B2042C08D82146154B03EB44139B68F9
S31508004500002BEAD10123E9E700240EE001231D4030
S315080045102046FFF7C3FF0F4B720103EB4611043128
S31508004520985802F03BFF0134E4B2032C0AD8264619
S31508004530084B03EB44139B68012BE8D0112BE5D0FD
S315080045400023E4E7284602B070BD00BF0010024011
S3150800455098D1000818D1000808B559B10B4B4FEA95
S31508004560401C03EB4010027F818853F80C0002F0D0
S31508004570F4FF08BD054B4FEA401C03EB4010027ED2
S31508004580818853F80C0002F0E8FFF2E718D100081A
S3150800459038B504460D4B420103EB4015A9889858D7
S315080045A002F0D4FFEB69012B07D0084B03EB441349
S315080045B09B69012B05D0002038BD0128F5D10120C3
S315080045C0FAE708B10020F7E70120F5E798D10008D7
S315080045D008B5044B420103EB40108188985802F055
S315080045E0C1FF08BD18D100080120704708B5002191
S315080045F01320FFF78DFA08BD08B501461320FFF70B
S3150800460087FA08BD00230BB10020704703EB83022D
S31508004610034951F822208242F6D00133DBB2F2E791
S3150800462038D2000808B5044805F0FEFC034B1860AC
S31508004630003818BF012008BD4CD2000860020020CF
S3150800464038B504460378244D03EB830305EB83034F
S315080046504FF0FF31586805F0DBFD237803EB830341
S3150800466005EB8303D96841F002011C4B186805F075
S315080046702AFD237803EB8300A389A268616855F8AD
S31508004680200004F043F900280CBF0125002511D0AD
S315080046900020237810F0020F05F0010518BF002549
S315080046A003EB83030C4A02EB8303586805F0DFFD2E
S315080046B0284638BD237803EB8303074A02EB8303B6
S315080046C0D9684FF0FF33002241F002010348006821
S315080046D005F019FDDDE700BF38D2000860020020AA
S315080046E008B5FFF78FFF00EB8000044B03EB800350
S315080046F0D968034B186805F0B9FC08BD38D200081C
S315080047006002002008B5FFF77DFF00EB8000044B30
S3150800471003EB8003D968034B186805F0A7FC08BDAE
S3150800472038D200086002002010B50446006E40F03A
S315080047300070FFF761FF2046FFF764FF0221024B76
S31508004740186805F093FC10BD6002002007EE900A79
S31508004750F8EEE77A9FED097A87EE870ADFED087AA1
S3150800476060EE277A9FED077A77EE877A20EE270A9A
S31508004770DFED057A30EE670A704700BFECB9FE45F3
S31508004780DB8A1F416DE76B4342E0754310B584B081
S3150800479000238DF80F300A2005F0CAFB01248FE0AC
S315080047A09DF80F0010F0010F2CD010F0800F05D1E6
S315080047B010F0400F05D0544B01932BE0534B019357
S315080047C028E010F0200F08D04F4B019340F0A4606A
S315080047D040F48020FFF710FF1CE010F0100F02D005
S315080047E0494B0193F2E710F0080F02D0464B0193AC
S315080047F0ECE710F0040F02D0434B0193E6E7424B77
S315080048000193E3E710F0020F09D03F4B01934048AC
S31508004810FFF7F2FE00238DF80F3001245FE03A4BD4
S3150800482001933C48FFF7E8FEF4E79DF80F0010F007
S31508004830010F2CD010F0800F05D110F0400F05D0D5
S31508004840314B02932BE0314B029328E010F0200FF6
S3150800485008D02D4B029340F0A26040F48020FFF769
S31508004860CBFE1CE010F0100F02D0274B0293F2E7A4
S3150800487010F0080F02D0244B0293ECE710F0040F57
S3150800488002D0214B0293E6E71F4B0293E3E710F0B1
S31508004890020F33D01C4B02931F48FFF7ADFE0023CF
S315080048A08DF80F3001249DED010A0820FFF734F931
S315080048B09DED020A0920FFF72FF9642005F038FB61
S315080048C003AA0DF10F010020FFF746FA04403FF452
S315080048D067AFBDF80C00FFF739FF8DED010A03AA93
S315080048E00DF10F010120FFF737FA04409DD0BDF8FE
S315080048F00C00FFF72BFF8DED020AD4E7024B02935B
S315080049000648FFF779FECAE77B9488C300408345CB
S31508004910000021050000220500001105000012050F
S3150800492008B5054A0021054805F099FA044B1860B0
S31508004930003818BF012008BD6CD200088D47000852
S315080049406402002008B504F03BFDB0FA80F0400987
S3150800495008BD70B505460E4605F0F6F9044610F48E
S31508004960807F04D10120E4B2FF2C0ED070BD04F084
S3150800497045FB0443A4B23146284605F0E5F9204331
S3150800498080B2B0FA80F04009EDE70020EEE70000BB
S3150800499010B502F09FFBB0FA80F46409024B186860
S315080049A005F065FC204610BD6802002008B54FF0EA
S315080049B0FF31054B186805F02BFC02F073FBB0FAC3
S315080049C080F0400908BD00BF6802002010B50B48FA
S315080049D005F0D3FB0A4B1860041E18BF0124FFF725
S315080049E0E5FF0440002004F0A5FE002814BF0024BB
S315080049F004F00104FFF7CCFF204010BD90D2000858
S31508004A0068020020014A024B9A6070470028000895
S31508004A1000ED00E02DE9F04188B0002403940494E9
S31508004A20059406940794364BDA6C42F00402DA646D
S31508004A30DA6C02F004020092009ADA6C42F0010283
S31508004A40DA64DA6C02F001020192019ADA6C42F039
S31508004A500202DA64DB6C03F002030293029B294F1D
S31508004A6022464FF48041384602F077FD22464FF43D
S31508004A7080714FF0904002F070FD234D2246602170
S31508004A80284602F06AFD4FF48043039301260496F4
S31508004A900594069403A9384602F080FC4FF40048B2
S31508004AA0CDF80C800494059403A9384602F076FCE8
S31508004AB04FF48073039304960594069403A94FF064
S31508004AC0904002F06BFCCDF80C800494059403A981
S31508004AD04FF0904002F062FC9823039304940594E7
S31508004AE003A9284602F05AFC60230393049605940A
S31508004AF0069403A9284602F051FC08B0BDE8F081E7
S31508004B0000100240000800480004004800B583B0C1
S31508004B10164B9A6C42F001029A649A6C02F00102F2
S31508004B200092009A9A6C42F002029A649B6C03F017
S31508004B3002030193019B002205210C2001F0F4FEDB
S31508004B400C2001F001FF002205210D2001F0ECFEEA
S31508004B500D2001F0F9FE002205213A2001F0E4FEBD
S31508004B603A2001F0F1FE03B05DF804FB00100240A4
S31508004B7008B5FEF739FC024B186805F0CAF9FEE7D6
S31508004B806C02002008B50020FEF78CFD01F0E0FE5F
S31508004B9072B6FEE700B587B000230093019302932F
S31508004BA00393049305932F482F4A0260436083605A
S31508004BB0C36001220261082141610376427604211D
S31508004BC0C16180F820308362C36280F83020436375
S31508004BD080F838201C21C163802101644364826403
S31508004BE000F09EFC002832D1204B00930623019347
S31508004BF0072302937F230393042304930023059337
S31508004C006946184800F0E2FE18BB194B00930C23BE
S31508004C1001936946134800F0D9FEE0B9154B009395
S31508004C201223019369460F4800F0D0FEA8B9124B2B
S31508004C3000931823019369460A4800F0C7FE70B925
S31508004C407F21084801F0F2F907B05DF804FBFFF789
S31508004C5099FFFFF797FFFFF795FFFFF793FFFFF71A
S31508004C6091FF00BF70040020000004504000201986
S31508004C70000021438000501D0080F03E08B50D4815
S31508004C800D4B03602023436000238360C3604FF409
S31508004C90402202614FF4A00242610376437683768E
S31508004CA00122C2760377437701F011FA00B908BDED
S31508004CB0FFF768FF000400200064004000B58BB0D1
S31508004CC02422002101A807F0F6FE1048104B0360C5
S31508004CD001F0D2FE98B90022019202920392049240
S31508004CE0059201A9094801F022FF50B9002201A93D
S31508004CF0064801F0C1FF30B90BB05DF804FBFFF7B9
S31508004D0041FFFFF73FFFFFF73DFF00BFC803002045
S31508004D100074004008B51048104B03604FF48273C6
S31508004D204360002383604FF4E062C260036101229E
S31508004D3042614FF4007282613022C26103624362AB
S31508004D4083620722C2620363436303F06FFD00B9FF
S31508004D5008BDFFF717FF00BF000300200030014021
S31508004D6008B51148114B0360114B4360002383605B
S31508004D700122C260036143618361C361036202F079
S31508004D80FAFB50B90021084802F059FC38B900214D
S31508004D90054802F082FC20B908BDFFF7F3FEFFF7CD
S31508004DA0F1FEFFF7EFFE00BF740300200054004039
S31508004DB0E49CD11008B50848084B036006234360F5
S31508004DC040F6FF73C3609623836002F092FC00B935
S31508004DD008BDFFF7D7FE00BF64030020003000407F
S31508004DE008B50848084B0360002303714371436103
S31508004DF083610123036201F0C3FD00B908BDFFF713
S31508004E00C1FE00BFDC0300200030024000B597B0A9
S31508004E104422002105A807F04EFE002300930193C3
S31508004E200293039304934FF4007002F0A7FC30BB7F
S31508004E30092305934FF4A023069301230A9302231B
S31508004E400F93032210920422119210221292072223
S31508004E5013921493159305A802F074FD88B90F23CD
S31508004E6000930323019300230293039304930421DD
S31508004E70684603F09DF830B917B05DF804FBFFF7F4
S31508004E8081FEFFF77FFEFFF77DFE000008B5FFF7FE
S31508004E90B9FD00F0E1FAFFF7B9FFFFF7BBFDFFF731
S31508004EA035FEFFF777FEFFF7E9FEFFF707FFFFF787
S31508004EB031FFFFF755FFFFF77DFFFFF791FF04F07E
S31508004EC08BFF054A0021054804F0C9FF044B18600A
S31508004ED004F094FFFEE700BFA0D20008714B00085B
S31508004EE06C02002000B583B00D4B1A6E42F0010229
S31508004EF01A661A6E02F001020092009A9A6D42F042
S31508004F0080529A659B6D03F080530193019B0022A2
S31508004F100F216FF0010001F007FD03B05DF804FBF7
S31508004F200010024070B59EB00446002119911A91EE
S31508004F301B911C911D91542204A807F0BCFD226800
S31508004F40334B9A4201D01EB070BD4FF48043049390
S31508004F504FF04053169304A803F0A6F9002850D141
S31508004F602C4BDA6C42F40052DA64DA6C02F4005222
S31508004F700192019ADA6C42F00102DA64DA6C02F004
S31508004F8001020292029ADA6C42F00202DA64DB6CDF
S31508004F9003F002030393039B062319930B261A9621
S31508004FA000251B9519A94FF0904002F0F7F9032345
S31508004FB019931A961B9519A9174802F0EFF917487D
S31508004FC0174B036045608560C560802303614FF415
S31508004FD0807343614FF4806383612023C3614FF478
S31508004FE00053036201F0F0FE70B90C4BE3649C6257
S31508004FF000220521122001F097FC122001F0A4FCE2
S31508005000A1E7FFF7BFFDABE7FFF7BCFDEDE700BF84
S315080050100000045000100240000400482804002044
S315080050203004024000B589B0002303930493059326
S31508005030069307930268244B9A4202D009B05DF89A
S3150800504004FB03F5D6339A6D42F000729A659A6DA1
S3150800505002F000720192019ADA6C42F00102DA64F7
S31508005060DB6C03F001030293029B4FF4C0530393D6
S3150800507002230493032306930923079303A94FF0F6
S31508005080904002F08BF900220521132001F04CFC18
S31508005090132001F059FC00220521142001F044FCDC
S315080050A0142001F051FC00220521152001F03CFCDA
S315080050B0152001F049FC00220521162001F034FCD8
S315080050C0162001F041FCB9E7006400400268094B6C
S315080050D09A4200D0704782B0A3F500539A6C42F406
S315080050E080529A649B6C03F480530193019B02B02F
S315080050F0704700BF0030024000B589B00023039313
S3150800510004930593069307930268124B9A4202D0BA
S3150800511009B05DF804FB03F5CE339A6D42F00052F0
S315080051209A659A6D02F000520192019ADA6C42F081
S315080051300102DA64DB6C03F001030293029B10237D
S3150800514003930323049303A94FF0904002F026F932
S31508005150DEE700BF0074004010B59CB0044600218D
S315080051601791189119911A911B91542202A807F0C8
S31508005170A2FC2268184B9A4201D01CB010BD4023ED
S31508005180029302A803F090F818BB144CE36C43F0A2
S315080051900103E364E36C03F001030093009B4FF4FF
S315080051A0C0631793122318930023199303231A93A2
S315080051B004231B9317A94FF0904002F0EFF8A36D54
S315080051C043F40013A365A36D03F400130193019B35
S315080051D0D3E7FFF7D7FCD8E7005400400010024099
S315080051E010B588B000230393049305930693079399
S315080051F002682F4B9A4201D008B010BD044603F549
S3150800520060431A6E42F480521A661A6E02F480528D
S315080052100192019ADA6C42F00102DA64DB6C03F05F
S3150800522001030293029BE0230393022304930323BF
S3150800523006930523079303A94FF0904002F0AEF8B2
S315080052401C481D4B03600123436000238360C36031
S315080052508022026143618361C361036201F0B4FD88
S3150800526000BB144BA3659C621448154B03600123CD
S315080052704360102383600023C36080220261436178
S315080052808361C361036201F09FFD70B90B4B6365CF
S315080052909C6200220521232001F046FB232001F011
S315080052A053FBA9E7FFF76EFCDBE7FFF76BFCEDE7BF
S315080052B000300140B80200201C00024070020020A5
S315080052C03000024008B50020FEF7ECF901F040FB7B
S315080052D0FEE708B50020FEF7E5F901F039FBFEE721
S315080052E008B50020FEF7DEF901F032FBFEE708B547
S315080052F00020FEF7D7F901F02BFBFEE708B50020E2
S31508005300FEF7D0F901F024FBFEE7704708B500F078
S31508005310B3F806F0FBFC012800D108BD07F09AF99E
S31508005320FBE7000008B5024801F033FE08BD00BFE0
S31508005330B802002008B5024801F02BFE08BD00BFE0
S315080053407002002008B5024800F0D4F908BD00BF75
S315080053507004002008B5024801F057F908BD00BFDF
S315080053600004002008B5024801F04FF908BD00BF47
S315080053700004002008B5024801F047F908BD00BF3F
S315080053800004002008B5024801F03FF908BD00BF37
S315080053900004002008B5024803F048FC08BD00BF19
S315080053A00003002008B5024801F0F3FD08BD00BF60
S315080053B0280400200E4AD2F8883043F47003C2F855
S315080053C088300C4B1A6842F001021A600021996075
S315080053D01A6822F0A85222F410221A604FF480525A
S315080053E0DA601A6822F480221A609961704700BF51
S315080053F000ED00E00010024008B50B4601461846CD
S3150800540007F0E6FB08BD0000104B1B780BB901201E
S31508005410704710B504464FF47A70B0FBF3F30C4AA4
S315080054201068B0FBF3F001F097FA68B90F2C01D9B0
S3150800543001200AE0002221464FF0FF3001F074FAFD
S31508005440044B1C60002000E0012010BD98000020DD
S31508005450940000209C00002010B5032001F052FAA9
S315080054600F20FFF7D1FF10B10124204610BD0446D6
S31508005470FFF738FDF9E70000034B1B78034A11686C
S315080054800B441360704700BF98000020D404002026
S31508005490014B1868704700BFD404002038B504468D
S315080054A0FFF7F6FF0546B4F1FF3F02D0044B1B7821
S315080054B01C44FFF7EDFF401BA042FAD338BD00BFDE
S315080054C09800002010B430300B0A9B0003F00C0340
S315080054D0C45801F01F014FF01F0C0CFA01FC24EA16
S315080054E00C0CC2F384628A404CEA0202C2505DF890
S315080054F0044B704710B414304B0E9B0003F00403A2
S31508005500C458C1F304514FF0070C0CFA01FC24EA05
S315080055100C0C8A404CEA0202C2505DF8044B7047F4
S3150800552030B583B000230193002800F0D0800446EC
S31508005530436D13B323689A6812F0005F05D09A6822
S3150800554022F0204222F03F029A602268936813F004
S31508005550805F1FD1936823F0104323F03F0343F085
S31508005560805393605B4B1B689B095B4AA2FB032332
S315080055709B0901335B00019309E0FFF7D3FC002385
S31508005580A36584F85030D5E7019B013B0193019B45
S31508005590002BF9D12268936813F0805F70D1636D90
S315080055A043F010036365A36D43F00103A36501206F
S315080055B0936813F0040300D00123616D11F0100FF6
S315080055C07ED1002B7CD1636D23F4817343F00203F3
S315080055D06365936813F0010F0BD1404B9B6813F07A
S315080055E0010F06D163683E498A6822F47C12134388
S315080055F08B60627E636B43EA4233E2681343A268B8
S31508005600134394F8202043EA0243012A3AD0A26AB7
S3150800561022B102F47072E16A0A4313432168CD6825
S31508005620304A2A401A43CA602268936813F008036E
S3150800563000D00123ABB9237E94F83010490041EA23
S315080056408331D36823F4804323F002030B43D360EA
S3150800565094F83830012B1AD02268136923F0010315
S3150800566013612369012B22D02268136B23F00F03E1
S315080056701363636D23F0030343F00103636524E0BA
S31508005680002095E7626A013A43EA4243BFE7216888
S315080056900B696FF38A03E26B256C2A43656C2A4310
S315080056A0A56C2A43134343F001030B61D9E721682C
S315080056B00B6B23F00F03E269013A13430B63D8E738
S315080056C0636D43F010036365012003B030BD01200C
S315080056D0FBE700BF94000020632D3E050000045040
S315080056E00003045007C0F0FF08B5806AFEF7FEFC09
S315080056F008BD704770B5044603681E685D6816F0F5
S31508005700020F10D015F0020F0DD0436D13F0100FD5
S3150800571003D1436D43F400634365204600F0D6FC8D
S31508005720236802221A6016F0040F02D015F0040F3F
S3150800573005D116F0080F3AD015F0080F37D0636D6B
S3150800574013F0100F03D1636D43F400736365236888
S31508005750DA6812F4406F24D1DA6812F4005F20D1B7
S315080057601A6812F0080F1CD09A6812F0040F10D1AC
S315080057705A6822F00C025A60636D23F480736365DD
S31508005780636D13F4805F0CD1636D43F001036365A9
S3150800579007E0636D43F010036365A36D43F00103EF
S315080057A0A3652046FEF798FC23680C221A6016F0BB
S315080057B0200F02D015F0200F05D116F0400F4CD05F
S315080057C015F0400F49D0636D13F0100F03D1636DC8
S315080057D043F4005363652368DA6C12F0C00F2AD1CC
S315080057E00121DA6812F4406F27D10120DA6871B313
S315080057F012F0007F03D050B312F4005F27D1196866
S3150800580011F0400F23D012F4001F20D19A6812F02D
S31508005810080F14D15A6822F060025A60636D23F4A7
S3150800582080536365636D13F4807F10D1636D43F015
S31508005830010363650BE00021D3E70020D6E7636D1B
S3150800584043F010036365A36D43F00103A365204687
S3150800585000F038FC236860221A6016F0800F02D028
S3150800586015F0800F2DD116F4807F02D015F4807FB5
S3150800587032D116F4007F02D015F4007F38D116F025
S31508005880100F17D015F0100F14D0636B23B12368CF
S31508005890DB6813F0010F0AD0636D43F48063636518
S315080058A0A36D43F00203A3652046FEF729FC23688F
S315080058B010221A6016F4806F02D015F4806F23D177
S315080058C070BD636D43F4803363652046FFF711FFAF
S315080058D0236880221A60C6E7636D43F40033636564
S315080058E0204600F0F1FB23684FF480721A60C0E787
S315080058F0636D43F480236365204600F0E6FB236866
S315080059004FF400721A60BAE7636D43F48043636527
S31508005910A36D43F00803A36523684FF480621A60F9
S31508005920204600F0D0FBCBE708B50346806A426DF7
S3150800593012F0500F30D1436D43F40073436503688A
S315080059401A6812F0080F14D0DA6812F4406F20D1E2
S31508005950DB6813F4005F1CD1436D23F48073436541
S31508005960436D13F4805F14D1436D43F0010343651F
S315080059700FE0DB6813F0020F0BD1436D23F480733D
S315080059804365436D13F4805F03D1436D43F0010310
S315080059904365FEF7A1FB08BD426D12F0100F04D156
S315080059A0C26C526B18469047F5E7FEF7A9FBF2E77B
S315080059B008B5806A436D43F040034365836D43F041
S315080059C004038365FEF79CFB08BD0000F0B583B0B1
S315080059D00023019390F85030012B00F0048204460E
S315080059E00D46012380F850300068836813F0040FD1
S315080059F009D0636D43F0200363650120002384F812
S31508005A00503003B0F0BD4968052907D80239032983
S31508005A104ED8DFE801F0024F484A0C212A68FFF702
S31508005A2051FD2068836813F0040300D001238268BF
S31508005A3012F0080200D001220BB9002A3CD02268D5
S31508005A40936813F0010F17D12B68E868D2F8B010E5
S31508005A50C3F3120621EA060100F0180CA84820FA3A
S31508005A600CF00340C3F312030B43C2F8B030EA68E4
S31508005A70A44B9A4200F0A5802B68A34A134200F073
S31508005A80AE81A24A926802F0E070A1498B4200F00A
S31508005A905881A0498B4200F07B819F498B4200F0D8
S31508005AA08B810020AAE71821B8E74FF48071B5E783
S31508005AB00621B3E71221B1E7AA682968FFF71AFD9C
S31508005AC069692268D368C3F3C1035B0099402869F2
S31508005AD004280ED02E68603252F820708F4B3B4057
S31508005AE006F0F84631430B4343F0004342F82030B2
S31508005AF0A5E7136E116EC1F384612B68C3F3120018
S31508005B0080BBC3F38463994234D021684B6E4A6ED6
S31508005B10C2F384622B68C3F3120080BBC3F38463A9
S31508005B209A4234D021688B6E8A6EC2F384622B68DF
S31508005B30C3F3120080BBC3F384639A4234D021684E
S31508005B40CB6ECA6EC2F384622B68C3F3120080BBA5
S31508005B50C3F384639A427FF472AFCB6E23F000439B
S31508005B60CB666CE793FAA3F313B1B3FA83F3CAE7E8
S31508005B702023C8E7136E23F000431366C5E793FA9C
S31508005B80A3F313B1B3FA83F3CAE72023C8E74B6E2E
S31508005B9023F000434B66C5E793FAA3F313B1B3FAB0
S31508005BA083F3CAE72023C8E78B6E23F000438B668E
S31508005BB0C5E793FAA3F313B1B3FA83F3CAE720232D
S31508005BC0C8E720682B68C3F312063EBB9A0E01325B
S31508005BD002F01F02092A8CBF00220122002A55D092
S31508005BE05EBB990E0131890601F0F8418EBB4FEA7A
S31508005BF0936C0CF1010C0CF01F0C012202FA0CF24A
S31508005C001143AEBB9B0E013303F01F0303EB4303A3
S31508005C101B051943AA68FFF76DFC2DE793FAA3F253
S31508005C204AB1B2FA82F2013202F01F02092A8CBF87
S31508005C3000220122D2E72022F5E793FAA3F131B137
S31508005C40B1FA81F10131890601F0F841CEE7202148
S31508005C50F8E793FAA3F24AB1B2FA82F2013202F0F5
S31508005C601F024FF0010C0CFA02F2C9E72022F5E7F1
S31508005C7093FAA3F343B1B3FA83F3013303F01F0393
S31508005C8003EB43031B05C4E72023F6E7E6B9990EA1
S31508005C900131890601F0F84116BB4FEA936C0CF105
S31508005CA0010C0CF01F0C012202FA0CF21143BEBBC8
S31508005CB09B0E013303F01F0303EB43031E3B1B0537
S31508005CC043F000731943A5E793FAA3F131B1B1FA8A
S31508005CD081F10131890601F0F841DDE72021F8E775
S31508005CE093FAA3F24AB1B2FA82F2013202F01F0223
S31508005CF04FF0010C0CFA02F2D8E72022F5E700BFB4
S31508005D00FFFF070000007F400000088000030450E2
S31508005D10000052C7000084CB0100008000F0FF039A
S31508005D2093FAA3F35BB1B3FA83F3013303F01F03CA
S31508005D3003EB43031E3B1B0543F00073C2E7202316
S31508005D40F3E712F4000F7FF4A4AE2268274B9A42B9
S31508005D5001D0002052E640F4000325498A6822F063
S31508005D60E07213438B60234B1B689B09224AA2FBF4
S31508005D7003239B09013303EB43039B00019302E0D2
S31508005D80019B013B0193019B002BF9D1002035E6CD
S31508005D9012F0807F7FF481AE2268144B9A4201D0BC
S31508005DA000202BE640F0807311498A6822F0E072E1
S31508005DB013438B60002021E612F4800F11D122686C
S31508005DC00A4B9A4201D0002018E640F4800308499D
S31508005DD08A6822F0E07213438B6000200EE60020EA
S31508005DE00CE600200AE602200BE600BF000004507D
S31508005DF00003045094000020632D3E0530B583B09F
S31508005E000023019303689A6812F0010F58D10446DB
S31508005E1099682D4A114219D19A6822F0004222F057
S31508005E203F0242F001029A60284B9B6813F4000F68
S31508005E301CD0274B1B689B09264AA2FB03239B09F8
S31508005E40013303EB43039B0001930CE0436D43F0DE
S31508005E5010034365836D43F001038365012030E039
S31508005E60019B013B0193019B002BF9D1FFF710FB26
S31508005E70054623681A6812F0010F1FD19A6812F0B6
S31508005E80010F07D19A6822F0004222F03F0242F041
S31508005E9001029A60FFF7FCFA431B022BE9D9236833
S31508005EA01B6813F0010FE4D1636D43F010036365BB
S31508005EB0A36D43F00103A365012002E0002000E082
S31508005EC0002003B030BD00BF3F000080000304502F
S31508005ED094000020632D3E0570B50446006880686E
S31508005EE010F0040F4ED10E46154694F85030012B8B
S31508005EF04AD0012384F850302046FFF77FFF002858
S31508005F003CD1636D23F4706323F0010343F480737B
S31508005F106365636D13F4805F2DD0A36D23F00603CC
S31508005F20A365E36C194ADA62E36C194A1A63E36CEF
S31508005F30184A5A6323681C221A60002384F85030D2
S31508005F402268536843F0100353602268D36843F00D
S31508005F500103D36021682B4632464031E06C00F0DD
S31508005F60B5FF2268936823F0004323F03F0343F00C
S31508005F700403936007E00023A365D2E7002384F8AF
S31508005F80503000E0022070BD0220FCE729590008C5
S31508005F90E9560008B159000838B5044602689368FE
S31508005FA013F0020300D00123916811F0010F39D0D4
S31508005FB0002B39D1936803F00D03012B09D0636DCB
S31508005FC043F010036365A36D43F00103A365012045
S31508005FD029E0936823F0004323F03F0343F00203CC
S31508005FE09360236803221A60FFF752FA054623686E
S31508005FF09B6813F0010F13D0FFF74AFA401B0228DB
S31508006000F5D923689B6813F0010FF0D0636D43F050
S3150800601010036365A36D43F00103A365012002E045
S31508006020002000E0002038BD0020FCE730B583B032
S315080060300023019390F85030012B41D004460D46B9
S31508006040012380F85030FFF7A7FF80BB636D23F468
S31508006050885323F0020343F00203636522689368BA
S3150800606023F0404323F03F0305F080452B4343F0DC
S315080060700043936023689B68002B06DB636D23F05F
S31508006080030343F00103636515E0019B01330193A4
S31508006090019BB3F5912FEDD3636D23F0120343F003
S315080060A010036365002384F85030012006E0636D11
S315080060B043F010036365002384F8503003B030BD05
S315080060C00220FBE770477047704770477047002803
S315080060D000F0A18038B5044690F82030D3B1226884
S315080060E0136843F001031360FFF7D2F905462368E6
S315080060F05A6812F0010F10D1FFF7CAF9401B0A2897
S31508006100F5D9636A43F400336362052384F82030C3
S31508006110012038BDFEF786FFE1E71A6822F0020281
S315080061201A60FFF7B5F9054623685A6812F0020F98
S315080061300DD0FFF7ADF9401B0A28F5D9636A43F479
S3150800614000336362052384F820300120E1E7227ECC
S31508006150012A3DD01A6822F080021A60637E012B5C
S315080061603BD02268136823F040031360A37E012BFB
S3150800617039D02268136823F020031360E37E012BCD
S3150800618037D02268136843F010031360237F012B6E
S3150800619035D02268136823F008031360637F012B48
S315080061A033D02268136823F004031360A368E268F7
S315080061B0134322691343626913436268013A2168EB
S315080061C01343CB6100206062012384F82030A0E7E6
S315080061D01A6842F080021A60C0E72268136843F022
S315080061E040031360C2E72268136843F02003136074
S315080061F0C4E72268136823F010031360C6E7226811
S31508006200136843F008031360C8E72268136843F06D
S3150800621004031360CAE701207047026890F820302B
S31508006220013BDBB2012B05D9436A43F48023436261
S315080062300120704730B4D2F8003243F00103C2F8A7
S3150800624000324B6903F01F03012000FA03F3D2F86A
S315080062501C026FEA030C20EA0300C2F81C02C86994
S31508006260B0B9D2F80C020CEA0000C2F80C028C880D
S315080062704869CD6844EA0544483042F830400C88FD
S3150800628048698D6844EA0544483002EBC00044601A
S31508006290C86901281BD0886980BBD2F804020CEAB9
S315080062A00000C2F80402086970BBD2F814020CEAAE
S315080062B00000C2F81402096A01292BD0D2F800326C
S315080062C023F00103C2F80032002030BC7047D2F830
S315080062D00C021843C2F80C028C8848690D6844EA17
S315080062E00544483042F830408C8948698D6844EA4C
S315080062F00544483002EBC0004460CCE7D2F80402FB
S315080063001843C2F80402CEE7D2F814021843C2F8BA
S315080063101402D0E7D2F81C120B43C2F81C32CDE7A0
S3150800632070B5044690F82050EDB2012D06D0436AA8
S3150800633043F4002343620125284670BD022380F8F2
S3150800634020300268136823F001031360FFF7A0F8F2
S31508006350064623685B6813F0010F0CD0FFF798F820
S31508006360831B0A2BF5D9636A43F40033636205235A
S3150800637084F82030E0E700256562DDE730B590F85F
S3150800638020C00468A4680CF1FF3C5FFA8CFCBCF1E1
S31508006390010F62D814F0E05F59D0C4F3016C0124F0
S315080063A004FA0CF41C608B68002B3DD10D68CB6891
S315080063B0046843EA45550CF118031B01E5500368C8
S315080063C00C690CF1180E03EB0E135C600B7D012BA8
S315080063D035D0D17993791B0443EA0163517943EAAD
S315080063E0012314790168234301EB0C11C1F88C31A0
S315080063F0D17893781B0443EA0163517843EA012371
S31508006400117802680B4302EB0C12C2F88831026855
S315080064100CF1180C4FEA0C1C52F80C3043F001032F
S3150800642042F80C3000201DE04C6843EAC403CC68EF
S3150800643023430CF11804240105682B51BFE70368B0
S3150800644003EB0E13596841F480715960C1E7436A3A
S3150800645043F400134362012004E0436A43F48023B3
S315080064604362012030BD90F820C00CF1FF3C5FFA72
S315080064708CFCBCF1010F00F2A58030B451B9046858
S31508006480E46814F0030F10D1436A43F4001343621F
S3150800649001207EE00468246914F0030F05D1436ADD
S315080064A043F400134362012073E0056801F11B04FD
S315080064B024012C5904F004049460002C6BD105685F
S315080064C001F11B0424012C59640D1460046801F1C0
S315080064D01B0C4FEA0C1C54F80C4004F00204D46060
S315080064E00468A444DCF8045015F0080F5BD00824AF
S315080064F01461046801F11B0C04EB0C146468C4F302
S3150800650007249461046804EB0C146468240C546131
S31508006510026802EB0112D2F8B8211A70026802EB7F
S315080065200112D2F8B821C2F307225A70026802EBA8
S315080065300112D2F8B821C2F307429A70026802EB38
S315080065400112D2F8B821120EDA70026802EB0112B3
S31508006550D2F8BC211A71026802EB0112D2F8BC21EA
S31508006560C2F307225A71026802EB0112D2F8BC2163
S31508006570C2F307429A71026802EB0112D2F8BC21F3
S31508006580120EDA71C1B90268D36843F02003D360EA
S31508006590002030BC7047056801F11B0424012C5902
S315080065A0E408546092E701F11B0504EB05146468DE
S315080065B004F00F0414619CE70268136943F0200392
S315080065C01361E5E7436A43F4802343620120704779
S315080065D090F82030013BDBB2012B05D9436A43F41E
S315080065E08023436201207047026853690B43536155
S315080065F0002070477047704770477047704770476C
S31508006600704770477047704770472DE9F84F054641
S3150800661003685C69D3F804809F68D3F80CA0D3F8A4
S315080066201090D3F818B014F001063BD017F0010605
S3150800663016D001229A6017F0020F08D117F0040F3E
S315080066400CD117F0080606D04FF4805608E0FFF77D
S31508006650D1FF002604E0FFF7D0FF01E04FF4006603
S3150800666017F4807F0DD02B684FF480729A6017F468
S31508006670007F40F0968017F4806F00F0968046F40D
S31508006680005617F4803F0DD02B684FF480329A607D
S3150800669017F4003F40F0938017F4802F00F09380A2
S315080066A046F4004614F0080F07D01AF0100F04D06D
S315080066B046F400762B681022DA6014F0040F03D033
S315080066C01AF0080F40F0898014F0020F05D02B68E5
S315080066D0DB6813F0030F40F0878014F0400F07D0F3
S315080066E019F0100F04D046F480662B6810221A6140
S315080066F014F0200F02D019F0080F79D114F0100FFA
S3150800670004D02B681B6913F0030F78D114F4003FEB
S3150800671002D018F0100F76D114F4803F02D018F08A
S31508006720080F77D114F4004F37D018F0040F31D082
S3150800673014F4807F04D01BF0010F01D046F0010647
S3150800674014F4007F04D01BF0020F01D046F00206B5
S3150800675014F4806F04D01BF0040F01D046F0040631
S3150800676014F4006F16D01BF0700B13D0BBF1400F5A
S3150800677066D056D8BBF1200F5CD0BBF1300F5CD089
S31508006780BBF1100F01D146F008062A68936923F079
S31508006790700393612B6804225A60002E56D1BDE817
S315080067A0F88F2846FFF727FF6BE717F4006F02D02C
S315080067B046F4804665E72846FFF720FF61E7284646
S315080067C0FFF71AFF6EE717F4002F02D046F480365B
S315080067D068E72846FFF713FF64E72B680822DA60A4
S315080067E02846FFF70DFF6FE72846FDF71DFE74E7FD
S315080067F02B6808221A612846FFF704FF7EE7284619
S31508006800FFF7FFFE82E72B6810225A602846FFF73B
S31508006810FAFE81E72B6808225A602846FFF7F4FE3D
S3150800682080E7BBF1500F0ED0BBF1600FADD146F437
S315080068308076AAE746F01006A7E746F02006A4E702
S3150800684046F04006A1E746F080069EE76B6A3343AA
S315080068506B622846FDF70AFEA1E70000002807DB61
S3150800686000F01F02400901239340024A42F82030F3
S31508006870704700BF00E100E0002808DB0901C9B243
S3150800688000F1604000F5614080F80013704700F0A1
S315080068900F000901C9B2014B1954704714ED00E005
S315080068A000B500F00700C0F1070CBCF1040F28BFC3
S315080068B04FF0040C031D062B0FD9C31E4FF0FF3EE5
S315080068C00EFA0CF021EA000199400EFA03FE22EABC
S315080068D00E0241EA02005DF804FB0023EEE7000021
S315080068E0BFF34F8F0549CA6802F4E062044B1343AD
S315080068F0CB60BFF34F8F00BFFDE700BF00ED00E0A0
S315080069000400FA05074AD36823F4E0631B041B0C4A
S31508006910000200F4E060034343F0BF6343F400332E
S31508006920D360704700ED00E010B50446054BD86803
S31508006930C0F30220FFF7B4FF01462046FFF79CFF8D
S3150800694010BD00BF00ED00E008B5FFF787FF08BDE2
S3150800695008B5FFF7C5FF00000138B0F1807F0BD2FC
S315080069604FF0E0235861054AF02182F823100020F1
S31508006970986107221A6170470120704700ED00E010
S31508006980002838D010B50446437F1BB3022363772B
S3150800699023791BBB2368194A5A612268936823F036
S315080069A018039360637913BB23684FF0FF321A61AB
S315080069B02268936823F0600361690B439360226839
S315080069C0936823F08003A1690B43936001236377DF
S315080069D0002010BD0377FEF779FBD7E7E268A168C8
S315080069E0204600F00DF80028DCD00120F1E72368E6
S315080069F022691A61DCE70120704700BFB71DC10490
S31508006A0011F0010F30D010B41F231C46013B34B1DE
S31508006A1003F01F0C21FA0CFC1CF0010FF5D0182A04
S31508006A2024D8DFE802F00F232323232323231D235F
S31508006A3023232323232319232323232323230D005B
S31508006A40062B17D80368596101688B6823F0180369
S31508006A5013438B6000200AE0072BF3D9012006E0D8
S31508006A600F2BEFD9012002E00120704701205DF8C5
S31508006A70044B70470120FAE770B110B50446037954
S31508006A8033B102232371002020610123237110BD35
S31508006A904371FEF731FBF4E7012070474279012A7A
S31508006AA02CD010B4034601224271022018711C68CA
S31508006AB0206801F0100C02FA0CF20243226089B930
S31508006AC019680A6802F03C02042A06D001221A71E3
S31508006AD0002058715DF8044B70474A6842F001027D
S31508006AE04A60F3E719680A6802F47012B2F5802F53
S31508006AF0ECD14A6842F002024A60E7E70220704792
S31508006B0010B483B0002401940068019051B901992A
S31508006B100A4408320192019A1360002003B05DF816
S31508006B20044B704701990A4414320192F3E7F8B509
S31508006B304379012B00F09E8004460D461646012334
S31508006B404371022303710B68042B33D02B69012B85
S31508006B5000F083802068C16B06F01002072393407B
S31508006B6021EA03012B68AE683343EE68334393404A
S31508006B700B43C363206803684FF48041914023EABE
S31508006B80010303602068016840F6FC73934021EA1C
S31508006B9003016B6893400B43036020680368C021B8
S31508006BA001FA02F223EA020303600123237100209B
S31508006BB06071F8BDFEF76CFC07469EB123685B6BF7
S31508006BC0002B43DAFEF764FCC01B0128F6D92368BC
S31508006BD05B6B002BF2DA236943F008032361032079
S31508006BE02071E6E723685B6B13F4004F10D0FEF7BD
S31508006BF04FFCC01B0128F5D923685B6B13F4004FC3
S31508006C00F0D0236943F00803236103202071D0E7FD
S31508006C100120FEF743FC2368AA691A642068836C7E
S31508006C2006F0100240F2FF31914023EA0103E969B8
S31508006C3091400B4383642068C36CFF21914023EA8B
S31508006C400103296A91400B43C3647FE70120FEF7DD
S31508006C5025FC2368AA695A64E0E721688A6B06F06E
S31508006C6010001F23834022EA03026B698340134303
S31508006C708B636FE702209CE7002800F085802DE9EA
S31508006C80F04F83B0894604460379DBB2022B7DD0E8
S31508006C904379012B7CD0012141710068C56B02F054
S31508006CA010070723BB4005EA030B0568B94025EA28
S31508006CB0010101602068C16B6FEA030A21EA030338
S31508006CC0C3632368019392B9019B08330193019B1F
S31508006CD04FF400621A60226813684FF4804808FA75
S31508006CE007F843EA080313600825102605E0019B08
S31508006CF014330193EBE72E446D089DB121688B6B25
S31508006D001F22BA4023EA020306FA07F213438B63EB
S31508006D100120FEF7C3FB23685B6B38EA0303EAD15D
S31508006D20761BE9E721688B6B1F22BA40D54323EA15
S31508006D30020306FA07F213438B630120FEF7AEFB44
S31508006D4023685A6B18EA020F08D11E2E06D8013698
S31508006D509A6B154006FA07F73D439D632268136848
S31508006D6023EA08031360C9F814600123C9F8103030
S31508006D702268D36B0AEA030A4AEA0B03D3630020A4
S31508006D80607103B0BDE8F08F012070470120F8E775
S31508006D900220F6E730B4446C04F01C0C012404FA13
S31508006DA00CF4056C6C60046863608368102B05D06E
S31508006DB0036899600368DA6030BC704703689A60B4
S31508006DC00368D960F8E70000002871D010B40346BC
S31508006DD00168384A914248D8374A0A443748A0FBDE
S31508006DE00202120992005A64354A1A64022283F88A
S31508006DF0252008686FF30E109A68DC6822431C6920
S31508006E0022435C6922439C692243DC6922431C6A4B
S31508006E10224302430A609A68B2F5804F1BD0196C68
S31508006E20274A91422CD0264AD2F8A814586C00F06A
S31508006E301C0C0F2000FA0CF021EA0001C2F8A81475
S31508006E40D2F8A81458685C6C04F01C0C00FA0CF014
S31508006E500143C2F8A8140020D863012283F825202C
S31508006E6083F824005DF8044B7047164A0A44134811
S31508006E70A0FB0202120992005A64134A1A64B5E783
S31508006E80D2F8A810586C00F01C0C0F2000FA0CF071
S31508006E9021EA0001C2F8A810D2F8A81058685C6C5C
S31508006EA004F01C0C00FA0CF00143C2F8A810D2E753
S31508006EB00120704707040240F8FFFDBFCDCCCCCCBB
S31508006EC000000240F8FBFDBF0004024038B5044646
S31508006ED090F82400012832D0012084F8240094F880
S31508006EE02500C0B2012804D0002384F824300220EB
S31508006EF038BD022084F825000020E063256828684C
S31508006F0020F0010028602046FFF744FF236B5BB1A1
S31508006F102268136843F00E0313602268136843F06F
S31508006F20010313600020E3E72268136823F00403D3
S31508006F3013602268136843F00A031360EDE7022022
S31508006F40D6E708B590F82530DBB2022B03D0042328
S31508006F50C363012008BD0268136823F00E0313609B
S31508006F600268136823F001031360436C03F01C03E3
S31508006F70016C012202FA03F34B6080F825200023F6
S31508006F8080F82430836B13B198470020E2E700208D
S31508006F90E0E738B5036C196804682568436C03F0A4
S31508006FA01C0304229A400A4215D015F0040F12D089
S31508006FB0236813F0200F03D1236823F0040323600A
S31508006FC0436C03F01C02016C042393404B60036B73
S31508006FD003B1984738BD02229A400A421CD015F0E0
S31508006FE0020F19D0236813F0200F06D1236823F067
S31508006FF00A032360012380F82530436C03F01C0242
S31508007000016C022393404B60002380F82430C36A46
S31508007010002BDFD09847DDE7082202FA03F30B427C
S31508007020D8D015F0080FD5D0236823F00E032360B7
S31508007030436C03F01C03016C012202FA03F34B6054
S31508007040C26380F82520002380F82430436B002B88
S31508007050C0D09847BEE7000010B4064C616941F0FD
S31508007060010161610260BFF36F8F43605DF8044BF5
S31508007070704700BF00200240094A536943F4802341
S315080070805361EFF3108C72B6402351F8042B40F885
S31508007090042B013B13F0FF03F7D18CF310887047DC
S315080070A000200240094B5B69002B01DB002070477A
S315080070B0064B074A9A6002F188329A605B69002B90
S315080070C001DB002070470120704700BF0020024006
S315080070D023016745034A536943F00043536100207F
S315080070E0704700BF0020024038B50446FEF7D0F9C5
S315080070F00546144B1B6913F4803F09D0B4F1FF3FD2
S31508007100F7D0FEF7C5F9401BA042F2D3032015E0DD
S315080071100C4B1B690C4A134009D10A4B1B6913F027
S31508007120010F0CD0074B01221A61002006E007491F
S315080071304A681A434A60034A1361012038BD002091
S31508007140FCE700BF00200240FAC30200A0000020AE
S315080071502DE9F0411646284A1278012A49D00446F4
S315080071600D469846244B01221A704CF25030FFF710
S31508007170BBFF074608BB204B00225A601F4B1B6803
S3150800718013F4806F1FD01D4A136823F480631360BD
S31508007190194B02221A77D4B1631E012B1ED900247B
S315080071A04CF25030FFF7A0FF074624B1134A536943
S315080071B023EA0403536100F047F80F4B00221A70C4
S315080071C03846BDE8F0810C4B00221A77E3E73246D1
S315080071D043462846FFF740FF0124E1E731462846A3
S315080071E0FFF74AFF022C01D00024D9E74FF4802488
S315080071F0D6E70227E4E700BFA000002000200240EF
S3150800720010F0010F04D0054A536943F00403536193
S31508007210024A536943F480335361704700200240A1
S31508007220084B5A6922F47E72C00000F4FF600243DC
S315080072305A615A6942F002025A615A6942F4803226
S315080072405A61704700200240164B1B7FDBB2012BA8
S3150800725001D0032B10D1144A116821F40071116072
S31508007260116841F400611160116821F40061116030
S31508007270116841F400711160023BDBB2012B03D99E
S31508007280084B00221A777047074B1A6842F4805257
S315080072901A601A6822F480521A601A6842F48062E8
S315080072A01A60EDE7A000002000200240F8B5394B2F
S315080072B01B78012B6BD004460E46364B01221A70FA
S315080072C04CF25030FFF710FF074600285AD1314BD1
S315080072D000225A60304B1B6813F4007F2FD02E4BC8
S315080072E01B6813F4806F26D02B4A136823F4806337
S315080072F01360284B03221A772368012B31D04FF0ED
S31508007300FF333360A568A368E2681344AB4237D9F4
S3150800731061682846FFF784FF4CF25030FFF7E4FE19
S315080073201D4A536923F47E7323F00203536107460B
S3150800733028BB0135E7E7174B01221A77DCE7164B1E
S315080073401B6813F4806F08D0134A136823F480630C
S315080073501360104B02221A77CEE70E4B00221A77DB
S31508007360CAE76068FFF74CFF4CF25030FFF7BCFEE7
S315080073700746094A536923F00403536100E0356060
S31508007380FFF762FF034B00221A703846F8BD022742
S31508007390FBE700BFA000002000200240F0B583B044
S315080073A0002362E085685E000324B44025EA0405EC
S315080073B0CC68B4402C438460456825EA0C054C68C3
S315080073C0C4F300149C402C4344605FE0DD08083594
S315080073D050F8254003F0070C4FEA8C0C4FF00F0EBF
S315080073E00EFA0CFE24EA0E0E0C6904FA0CF444EAB2
S315080073F00E0440F8254060E0022400E0002404FA68
S315080074000EF42C430CF1020C4C4D45F82C404C4C18
S31508007410A568D44325EA02064F6817F4801F01D0F1
S3150800742042EA0506464DAE60ED6804EA05064F6871
S3150800743017F4001F01D042EA0506414DEE606D685B
S3150800744004EA05064F6817F4003F01D042EA05062C
S315080074503B4D6E602D682C404E6816F4803F01D077
S3150800746042EA0504364A146001330A6832FA03F41C
S3150800747062D04FF0010C0CFA03FC1CEA0202F3D0AE
S315080074804C6804F00304013C012C8BD94C6804F0C9
S315080074900304032C0CD0C4685D004FF0030C0CFAEF
S315080074A005FC24EA0C0C8C68AC4044EA0C04C46065
S315080074B04C6804F00304022C88D004684FEA430E93
S315080074C04FF0030C0CFA0EFC24EA0C0C4C6804F082
S315080074D0030404FA0EF444EA0C0404604C6814F439
S315080074E0403FC1D0174C256E45F001052566246E30
S315080074F004F001040194019C4FEA930C0CF1020577
S315080075000E4C54F8255003F0030E4FEA8E0E0F2446
S3150800751004FA0EF425EA0405B0F1904F3FF46EAF75
S31508007520094CA04206D004F58064A0423FF464AF3B
S31508007530072464E7012462E703B0F0BD00000140B8
S315080075400004014000100240000400480369194283
S3150800755001D001207047002070470AB18161704749
S3150800756081627047436901EA030221EA030141EA9D
S3150800757002418161704700285FD010B5044690F833
S315080075804130002B48D0242384F841302268136800
S3150800759023F0010313606368226823F070631361A4
S315080075A02268936823F400439360E368012B38D07C
S315080075B0A368226843F404439360E368022B36D039
S315080075C02268536823F4006353602268536843F0C3
S315080075D0007343F4004353602268D36823F40043DE
S315080075E0D360236962691343A169226843EA0123C8
S315080075F0D360E369216A22680B4313602268136823
S3150800760043F00103136000206064202384F84130AE
S31508007610206384F8420010BD80F84030FDF79CFDD9
S31508007620B1E7A368226843F400439360C5E722687C
S31508007630536843F400635360C7E701207047034665
S3150800764090F84120D2B2202A23D190F84020012A6E
S3150800765021D0012280F84020242280F841200068A9
S31508007660026822F0010202601868026822F4805259
S315080076700260186802681143016019680A6842F0D6
S3150800768001020A60202283F84120002083F8400086
S3150800769070470220704702207047034690F8412041
S315080076A0D2B2202A21D190F84020012A1FD00122E7
S315080076B080F84020242280F841200068026822F0E1
S315080076C0010202601868026822F4706242EA012226
S315080076D0026019680A6842F001020A60202283F8EB
S315080076E04120002083F8400070470220704702209E
S315080076F07047002831D038B5044603684CF6CC42AA
S315080077001A60036845F255521A60036842685A605F
S31508007710036882689A60FDF7BBFE05462368DA6847
S3150800772012F0070F0DD0FDF7B3FE401B41F601031B
S315080077309842F3D92368DB6813F0070FEED00320CD
S3150800774005E01969E268914202D01A61002038BD45
S315080077504AF6AA221A600020F9E701207047036852
S315080077604AF6AA221A60002070470000024B1868E1
S3150800777000F4C060704700BF00700040B0F5007F9D
S315080077800FD01F4B1B6803F4C063B3F5806F34D06A
S315080077901B4A136823F4C06343F480631360002014
S315080077A07047174B1B6803F4C063B3F5007F20D0FE
S315080077B0134A136823F4C06343F400731360114B30
S315080077C01B68322202FB03F30F4AA2FB03239B0C1E
S315080077D0013300E0013B0A4A526912F4806F01D076
S315080077E0002BF7D1064B5B6913F4806F03D1002099
S315080077F0704700207047032070470020704700BF7D
S31508007800007000409400002083DE1B4330B583B02F
S315080078100446204B9B6D13F0805F0BD0FFF7A6FF45
S31508007820B0F5007F17D0802C1FD82DD0702C2DD006
S3150800783000211BE0174DAB6D43F08053AB65AB6D74
S3150800784003F080530193019BFFF790FFAB6D23F084
S315080078508053AB65E4E7802C03D9A02C03D9022119
S3150800786004E0002102E0012100E003210A4A13682E
S3150800787023F007030B431360136803F007038B42D7
S3150800788006D1002003B030BD0221EFE70121EDE764
S315080078900120F7E70010024000200240254A9368BD
S315080078A0D26802F0030213F00C0309D00C2B05D0A2
S315080078B0042B3BD0082B3BD000200FE0012AF7D140
S315080078C01C4A126812F0080F0CD11A4AD2F89420F2
S315080078D0C2F30322184951F8220013B10C2B06D023
S315080078E000207047134A1268C2F30312F2E7114BDD
S315080078F0DB6803F00303022B16D0032B00D10F48D5
S315080079000C49CA68C2F302120132CB68C3F30623D4
S3150800791000FB03F3B3FBF2F3C868C0F34160013020
S315080079204000B3FBF0F070470548E9E704487047A4
S315080079300248704700100240C4D20008005A62028A
S315080079400024F400002800F01C83F0B583B0044638
S31508007950964B9D6805F00C05DE6806F0030603687D
S3150800796013F0100F5AD0E5B10C2D18D0A369002BCF
S3150800797000F0BB808D4A136843F001031360FDF7DE
S3150800798087FD0746894B1B6813F0020F40F09A8063
S31508007990FDF77EFDC01B0228F4D90320FCE2012E68
S315080079A0E4D1824B1B6813F0020F03D0A369002BA6
S315080079B000F0E982206A7D4B1B6813F0080F5BD044
S315080079C07A4B1B6803F0F00398425CD8774B1A6829
S315080079D042F008021A601A6822F0F002216A0A4385
S315080079E01A605A6822F47F42E16942EA01225A6023
S315080079F0002D60D0FFF752FF6C4B9B68C3F303134F
S31508007A006B4AD35C03F01F03D8406A4B18606A4B75
S31508007A101868FDF7F9FC002840F0BE82236813F0C9
S31508007A20010F00F08180082D75D00C2D71D0636888
S31508007A30B3F5803F00F09780B3F5A02F00F099804A
S31508007A405A4B1A6822F480321A601A6822F4802285
S31508007A501A606368002B00F09980FDF719FD074648
S31508007A60524B1B6813F4003F5ED1FDF711FDC01B96
S31508007A706428F5D903208FE24C4BD3F894301B09C0
S31508007A8003F0F003A0E7FFF7C1FE002840F07D826F
S31508007A90464B1A6842F008021A601A6822F0F00289
S31508007AA0216A0A431A605A6822F47F42E16942EA67
S31508007AB001225A609EE7206AFFF7A8FE002899D09F
S31508007AC0012069E2394B1A6842F008021A601A68FE
S31508007AD022F0F002216A0A431A605A6822F47F42A9
S31508007AE0E16942EA01225A6098E7304A136823F0AE
S31508007AF001031360FDF7CCFC07462C4B1B6813F0FB
S31508007B00020F8BD0FDF7C4FCC01B0228F5D9032051
S31508007B1042E2032E8BD1254B1B6813F4003F03D09A
S31508007B206368002B00F03382236813F0020F58D0E5
S31508007B30042D45D00C2D41D0E368002B77D01B4A85
S31508007B40136843F480731360FDF7A2FC0646174BCF
S31508007B501B6813F4806F61D1FDF79AFC801B02281D
S31508007B60F5D9032018E2114A136843F480331360E9
S31508007B706FE703F18043A3F53C331A6842F4802289
S31508007B801A601A6842F480321A6062E7FDF780FCD0
S31508007B900746064B1B6813F4003FC5D0FDF778FC73
S31508007BA0C01B6428F5D90320F6E100BF0010024087
S31508007BB0F4D20008940000209C000020022EBBD1BD
S31508007BC0A44B1B6813F4806F03D0E368002B00F006
S31508007BD0E081A04A536823F0F853216943EA016318
S31508007BE05360236813F0080F4CD063699BB3994A16
S31508007BF0D2F8943043F00103C2F89430FDF748FCFC
S31508007C000646944BD3F8943013F0020F3AD1FDF799
S31508007C103FFC801B0228F4D90320BDE18D4A536836
S31508007C2023F0F853216943EA01635360D9E7894A87
S31508007C30136823F480731360FDF72AFC0646854B08
S31508007C401B6813F4806FCCD0FDF722FC801B02283A
S31508007C50F5D90320A0E17F4AD2F8943023F0010336
S31508007C60C2F89430FDF714FC06467A4BD3F89430E4
S31508007C7013F0020F06D0FDF70BFC801B0228F4D97F
S31508007C80032089E1236813F0040F7AD0714B9B6DAA
S31508007C9013F0805F36D16F4B9A6D42F080529A6529
S31508007CA09B6D03F080530193019B01266A4B1B6869
S31508007CB013F4807F28D0A368012B39D0052B3FD039
S31508007CC0644BD3F8902022F00102C3F89020D3F831
S31508007CD0902022F00402C3F89020A368002B3DD020
S31508007CE0FDF7D6FB07465B4BD3F8903013F0020F2F
S31508007CF046D1FDF7CDFBC01B41F288339842F2D935
S31508007D00032049E10026D1E7534A136843F48073F8
S31508007D101360FDF7BDFB07464F4B1B6813F4807FC6
S31508007D20C9D1FDF7B5FBC01B0228F5D9032033E1FD
S31508007D30484AD2F8903043F00103C2F89030CCE7B5
S31508007D40444BD3F8902042F00402C3F89020D3F8AD
S31508007D50902042F00102C3F89020BEE7FDF798FB99
S31508007D6007463C4BD3F8903013F0020F08D0FDF7C6
S31508007D708FFBC01B41F288339842F2D903200BE1EE
S31508007D80E6B9236813F0200F35D0636AE3B1314AA8
S31508007D90D2F8983043F00103C2F89830FDF778FB23
S31508007DA006462C4BD3F8983013F0020F23D1FDF773
S31508007DB06FFB801B0228F4D90320EDE0254A936D5A
S31508007DC023F080539365DCE7224AD2F8983023F0F3
S31508007DD00103C2F89830FDF75BFB06461D4BD3F846
S31508007DE0983013F0020F06D0FDF752FB801B0228CD
S31508007DF0F4D90320D0E0A36A002B00F0CC80022B34
S31508007E0017D00C2D00F0CC80124A136823F080732B
S31508007E101360FDF73DFB04460E4B1B6813F0007F0D
S31508007E2000F0A880FDF734FB001B0228F4D90320D4
S31508007E30B2E0084BDB6803F00301E26A91420DD019
S31508007E400C2D00F0AB80034B1B6813F0806F2FD00E
S31508007E500120A1E0001002400070004003F070020B
S31508007E60216B0139B2EB011FEAD103F4FE42616BC3
S31508007E70B2EB012FE4D103F07842A16BB2EBC16FEC
S31508007E80DED103F4C001E26B5208013AB1EB425F5E
S31508007E90D6D103F0C063226C5208013AB3EB426FA5
S31508007EA0CED1404B1B6813F0007F49D0002073E009
S31508007EB03C4A136823F080731360FDF7E9FA054618
S31508007EC0384B1B6813F0007F06D0FDF7E1FA401B1C
S31508007ED00228F5D903205FE0324AD36832491940AF
S31508007EE0E36A206B013843EA0013606B43EA002318
S31508007EF0E06B4008013843EA4053206C40080138DB
S31508007F0043EA4063A06B43EAC0631943D160136830
S31508007F1043F080731360D36843F08073D360FDF732
S31508007F20B7FA04461F4B1B6813F0007F06D1FDF70E
S31508007F30AFFA001B0228F5D903202DE000202BE01C
S31508007F40184B1A6842F080721A60DA6842F080723A
S31508007F50DA60FDF79DFA0446124B1B6813F0007FA2
S31508007F6006D1FDF795FA031B022BF5D9032013E07A
S31508007F70002011E00B4AD1680C4B0B40D36000205F
S31508007F800AE001207047012006E0012004E00120F4
S31508007F9002E0012000E0002003B0F0BD0120FBE76D
S31508007FA00120F9E7001002408C809D01FCFFEEFEDF
S31508007FB0002800F0AF8070B50D460446594B1B6883
S31508007FC003F007038B420BD2564A136823F00703C4
S31508007FD00B431360136803F007038B4240F09C8041
S31508007FE0236813F0020F0CD0A2684F4B9B6803F06E
S31508007FF0F0039A4205D94C498B6823F0F0031A43DB
S315080080008A60236813F0010F39D06368032B09D0FF
S31508008010022B26D063BB444A126812F0020F06D11F
S31508008020012076E0404A126812F0007F76D03E4979
S315080080308A6822F0030213438B60FDF729FA064685
S31508008040394B9B6803F00C036268B3EB820F16D0BA
S31508008050FDF71EFA801B41F288339842F0D90320B7
S3150800806057E0314A126812F4003FE0D1012050E08F
S315080080702D4A126812F4806FD9D1012049E023688D
S3150800808013F0020F0CD0A268274B9B6803F0F0038D
S315080080909A4205D224498B6823F0F0031A438A6072
S315080080A0204B1B6803F00703AB420AD91D4A136825
S315080080B023F007032B431360136803F00703AB424F
S315080080C02ED1236813F0040F06D0174A936823F4B9
S315080080D0E063E1680B439360236813F0080F07D049
S315080080E0114A936823F46053216943EAC1039360F4
S315080080F0FFF7D4FB0C4B9B68C3F303130B4AD35C03
S3150800810003F01F03D8400A4B18600A4B1868FDF79E
S315080081107BF970BD012070470120FAE70120F8E7D6
S315080081200120F6E70020024000100240F4D20008C1
S31508008130940000209C000020F8B504460D46594BD3
S31508008140DB6813F0030F18D0564BDB6803F0030304
S315080081500268934202D001263046F8BD002A00F094
S315080081609C80504BDB68C3F3021301334268934289
S3150800817001D00126F0E7002619E00368022B55D046
S31508008180032B5AD0012B40F08A80464A126812F017
S31508008190020F5ED04348C26822F073026168013953
S315080081A043EA01131343C3600026002ED4D13D4A87
S315080081B0136823F080631360FDF76AF90746394BA5
S315080081C01B6813F0006F05D0FDF762F9C31B022B7D
S315080081D0F5D90326002EBFD1002D3CD131490B69B4
S315080081E023F0784323F4FE43A068E268D20642EA05
S315080081F0002213430B612B4A136843F08063136014
S31508008200FDF746F90546274B1B6813F0006F05D1A5
S31508008210FDF73EF9401B0228F5D90326002E9BD10F
S31508008220204A1369A1690B43136195E71D4A126831
S3150800823012F4806FAED101268EE71A4A126812F43C
S31508008240003FA7D1174A126812F4802FA2D101263F
S3150800825082E70126A9E7012D0FD01248026922F00C
S31508008260C06222F4FE42A16863695B08013B5B06B3
S3150800827043EA01231A430261BDE70A48026922F468
S31508008280C00222F4FE42A16823695B08013B5B0534
S3150800829043EA01231A430261ADE701265CE701269A
S315080082A05AE700BF001002402DE9F04182B00446AB
S315080082B0036813F4006F26D0C36BB3F5000F06D01E
S315080082C0B3F5400F1DD09BB1012637461DE0AE4AD7
S315080082D0D36843F48033D3600027AB4AD2F888309A
S315080082E023F44003E16B0B43C2F8883000260CE008
S315080082F000210430FFF720FF07460028EDD0064688
S3150800830003E00027E9E700263746236813F4003F11
S315080083106BD09D4B9B6D13F0805F4CD19A4B9A6D39
S3150800832042F080529A659B6D03F080530193019B3E
S315080083304FF00108954A136843F480731360FDF7FC
S31508008340A7F80546914B1B6813F4807F05D1FDF706
S315080083509FF8401B0228F5D90327002F40D18A4BE6
S31508008360D3F8903013F4407318D0226D9A4212D085
S31508008370854AD2F8903023F44073D2F8901041F42D
S315080083808031C2F89010D2F8901021F48031C2F8EA
S315080083909010C2F8903013F0010F0FD1002F40F063
S315080083A0C980794AD2F8903023F44073216D0B4383
S315080083B0C2F8903015E04FF00008BBE7FDF768F803
S315080083C00546714BD3F8903013F0020FE6D1FDF74E
S315080083D05FF8401B41F288339842F2D90327DDE75C
S315080083E03E46B8F1000F40F0A780236813F0010F4E
S315080083F008D0654AD2F8883023F00303216A0B4374
S31508008400C2F88830236813F0020F08D05E4AD2F803
S31508008410883023F00C03616A0B43C2F8883023685E
S3150800842013F0200F08D0584AD2F8883023F4406356
S31508008430A16A0B43C2F88830236813F4007F08D07A
S31508008440514AD2F8883023F44023616B0B43C2F8B3
S315080084508830236813F4806F08D04B4AD2F88830E6
S3150800846023F44013A16B0B43C2F88830236813F03A
S31508008470400F08D0444AD2F8883023F44053E16AC2
S315080084800B43C2F88830236813F4807F08D03E4A2D
S31508008490D2F8883023F44033216B0B43C2F8883076
S315080084A0236813F4005F0FD0374AD2F8883023F0D8
S315080084B04063216C0B43C2F88830236CB3F1006F1C
S315080084C040D0B3F1806F42D0236813F4802F0FD0C9
S315080084D02D4AD2F8883023F04063616C0B43C2F80A
S315080084E08830636CB3F1006F39D0B3F1806F3BD03D
S315080084F0236813F4804F0CD0234AD2F8883023F02F
S315080085004053A16C0B43C2F88830A36CB3F1805F6B
S3150800851032D0236813F4004F08D01B4AD2F88830AB
S3150800852023F08043E16C0B43C2F88830304602B032
S31508008530BDE8F0813E4654E7134A936D23F0805315
S31508008540936552E7D36843F48013D360BCE70121EF
S31508008550201DFFF7F1FD0028B6D00646B4E7D3681C
S3150800856043F48013D360C3E70121201DFFF7E4FD20
S315080085700028BDD00646BBE70221201DFFF7DCFD1B
S315080085800028C6D00646C4E7001002400070004026
S315080085902DE9F04782B00546884617461E46FCF781
S315080085A077FF0A9B1B1A03EB0609FCF771FF824645
S315080085B0284B1B68C3F3CB3309FB03F301932B68E2
S315080085C09C6838EA04040CBF01230023BB423DD053
S315080085D0B6F1FF3FF3D0FCF75BFFA0EB0A00484576
S315080085E007D2019A02B14A46019B013B0193914683
S315080085F0E5E72A68536823F0E00353606B68B3F530
S31508008600827F0BD0AB6AB3F5005F14D0012385F8DF
S315080086105D30002385F85C30032018E0AB68B3F5BD
S31508008620004F02D0B3F5806FECD12A68136823F0A7
S3150800863040031360E6E72A68136823F400531360BF
S315080086402A68136843F400531360DFE7002002B07A
S31508008650BDE8F087940000202DE9F04782B0064671
S315080086600C4615461F4600238DF80330FCF710FF0D
S315080086700A9B1B1A03EB0708FCF70AFF8146D6F884
S3150800868000A0304B1B6803EB8303C3EBC3031B0D2E
S3150800869008FB03F3019302E0B7F1FF3F12D13368F9
S315080086A09B6803EA040CAC4547D0B4F5C06FF3D118
S315080086B0002DF1D19AF80C30DBB28DF803309DF815
S315080086C00330E9E7FCF7E4FEA0EB0900404507D2D2
S315080086D0019A02B14246019B013B01939046DEE7AF
S315080086E03268536823F0E00353607368B3F5827FFA
S315080086F00BD0B36AB3F5005F14D0012386F85D305A
S31508008700002386F85C30032018E0B368B3F5004F01
S3150800871002D0B3F5806FECD13268136823F04003BA
S315080087201360E6E73268136823F40053136032686F
S31508008730136843F400531360DFE7002002B0BDE876
S31508008740F08700BF9400002070B582B004460D463D
S31508008750164600920B4600224FF4C051FFF77CFFE5
S31508008760B0B900962B46002280212046FFF710FF5D
S31508008770A8B900962B4600224FF4C0612046FFF7A1
S315080087806BFF50B1236E43F020032366032004E0F9
S31508008790236E43F020032366032002B070BD236EC8
S315080087A043F0200323660320F7E770B582B004463A
S315080087B00D4616464368B3F5827F0DD000962B46C4
S315080087C0002280212046FFF7E3FE90B96368B3F5DF
S315080087D0827F14D002B070BD8368B3F5004F02D013
S315080087E0B3F5806FEAD12268136823F0400313605B
S315080087F0E4E7236E43F0200323660320EAE7A36831
S31508008800B3F5004F02D0B3F5806FE3D100962B463F
S3150800881000224FF4C0612046FFF71EFF0028D9D07A
S31508008820236E43F0200323660320D3E700286AD08B
S3150800883010B50446436A33B94368B3F5827F05D059
S315080088400023C36102E00023036143610023A3629E
S3150800885094F85D30002B4DD0022384F85D302268F1
S31508008860136823F040031360E368B3F5E06F47D954
S315080088700022B3F5706F04D0B3F5E06F01D0002382
S31508008880A362636803F48273A16801F404410B438D
S31508008890216901F002010B43616901F001010B43F3
S315080088A0A16901F400710B43E16901F038010B433A
S315080088B0216A01F080010B43A16A01F40051206886
S315080088C00B430360638B03F00403616A01F0100134
S315080088D00B43616B01F008010B43E16801F4706119
S315080088E00B43216813434B6000202066012384F85C
S315080088F05D3010BD84F85C302046FCF771FCABE7B0
S315080089004FF48052B5E701207047000038B5044699
S3150800891090F85D00C0B2656801280AD0B5F5827F77
S3150800892040F0E880A568002D40F0E680042840F075
S31508008930E580002900F0E480002A00F0E380002B9F
S3150800894000F0E28094F85C00012800F0DF80012046
S3150800895084F85C0094F85D00C0B2042802D00520B3
S3150800896084F85D0000202066A163A387E38722645C
S31508008970A4F84430A4F84630E064206522685368B9
S3150800898023F4C0435360E368B3F5E06F29D922683E
S31508008990536823F48053536094F85D30DBB2042B9C
S315080089A06AD0A36D5A4A1A63A36D5A4ADA62A36D4E
S315080089B0594A5A63A36D00229A632168B4F846306F
S315080089C09BB2226C0C31A06DFEF780FA00285AD0B3
S315080089D0236E43F010032366002384F85C300120DD
S315080089E089E02268536843F480535360636D9B693A
S315080089F0B3F5806F1AD0A36D9B69B3F5806FCBD1A1
S31508008A002268536823F480535360B4F8463013F051
S31508008A10010F24D12268536823F400535360B4F835
S31508008A204630C3F34E03A4F84630B5E7A38F13F0D8
S31508008A30010F09D12268536823F480435360E38FFA
S31508008A40C3F34E03E387D6E72268536843F48043AB
S31508008A505360E38FC3F34E030133E387CBE7226802
S31508008A60536843F400535360B4F84630C3F34E03D7
S31508008A700133A4F846308FE7A36D284A1A63A36D1D
S31508008A80274ADA6293E72268536843F00103536082
S31508008A90626D00231363626DD362626D5363626D08
S31508008AA093632268E38F9BB20C32A16B606DFEF76D
S31508008AB00DFAB0B923681A6812F0400F03D11A6884
S31508008AC042F040021A60002384F85C30226853683A
S31508008AD043F0200353602268536843F0020353604F
S31508008AE009E0236E43F010032366002384F85C3004
S31508008AF0012000E0022038BD0220FCE70220FAE748
S31508008B000120F8E70120F6E70120F4E70220F2E762
S31508008B10338B0008CF8B00083D8B0008278B000895
S31508008B205F8B0008704708B5806AFFF7FBFF08BD32
S31508008B30704708B5806AFFF7FBFF08BD08B5806A6D
S31508008B400268536823F003035360036E43F010036F
S31508008B500366012380F85D30FBF7E6FD08BD38B5EE
S31508008B600546846AFCF794FC2B681B6813F0200FF3
S31508008B701FD1024621684B6823F020034B60A36887
S31508008B801BB96368B3F5827F17D021684B6823F059
S31508008B9001034B6064212046FFF707FE08B1202336
S31508008BA023660023A4F84630012384F85D30236E3B
S31508008BB04BB92046FBF7A6FD38BD21684B6823F064
S31508008BC003034B60E6E72046FBF7AEFDF4E738B54E
S31508008BD00546846AFCF75CFC2B681B6813F0200FBB
S31508008BE01CD1024621684B6823F020034B606421A0
S31508008BF02046FFF7A9FD18B1236E43F0200323662C
S31508008C002268536823F0030353600023E387A4F81C
S31508008C104630012384F85D30236E1BB92046FBF7E6
S31508008C205FFD38BD2046FBF77FFDFAE730B585B016
S31508008C300446026851689368C3F3801013F0400F26
S31508008C4005D113F0010F02D011F0400F69D113F0CE
S31508008C50020F02D011F0800F67D1C3F3401513F04D
S31508008C60200F03D110B913F4807F61D011F0200FC3
S31508008C705ED078B194F85D00C0B203285AD0206E51
S31508008C8040F00400206600200090D06800909068AC
S31508008C900090009865B1206E40F001002066002023
S31508008CA0029090680290106820F040001060029AC6
S31508008CB013F4807F09D0236E43F00803236600234C
S31508008CC0039323689B680393039B236E002B2FD083
S31508008CD02268536823F0E0035360012384F85D306B
S31508008CE011F0030F2ED02268536823F00303536054
S31508008CF0A36D4BB1154A9A63A06DFEF722F918B118
S31508008D00236E43F040032366636D8BB10F4A9A6363
S31508008D10606DFEF716F958B1236E43F040032366DB
S31508008D2006E0E36C2046984702E0236D2046984704
S31508008D3005B030BD00230193D3680193936801936E
S31508008D40019BF5E72046FBF7EFFCF1E7518D00089C
S31508008D5008B5806A0023A0F84630C387FBF7E4FC11
S31508008D6008BD8446002311208B4212D230B402E09B
S31508008D7008338B420BD203EB0C02D2E90045B5F15E
S31508008D80FF3F08BFB4F1FF3FF2D01020F0E730BC38
S31508008D90704770472DE9F003D0E90089D0E90267EA
S31508008DA0D0E90445D0E90623B3F1FF3F08BFB2F185
S31508008DB0FF3F13D1B5F1FF3F08BFB4F1FF3F11D113
S31508008DC0B7F1FF3F08BFB6F1FF3F0DD1B9F1FF3F3D
S31508008DD008BFB8F1FF3F09D1002000E00420BDE834
S31508008DE0F00370470320FAE70220F8E70120F6E7C8
S31508008DF038B5044600F5803C4FEACC2C284BD3F80E
S31508008E00E02590B24FF6FF73984215D0254B03EA3A
S31508008E1082234FF4F032B2FBF3F203FB02CC0CF1DF
S31508008E2008050CF110000CF1180E0139032931D888
S31508008E30DFE801F005101B254FF48023E9E74FF022
S31508008E40AA324FF0AA33604600F08AFF20BB164BC1
S31508008E501C7038BD4FF0AA324FF0AA33284600F0EE
S31508008E607FFFD8B9104B1C70F3E74FF0AA324FF0CA
S31508008E70AA3300F075FF0028EBD00220E9E74FF08F
S31508008E80AA324FF0AA33704600F06AFF0028E0D0F5
S31508008E900220DEE70020DCE70220DAE70220D8E736
S31508008EA00070FF1F00FCFF03E004002038B50546EC
S31508008EB000F088FF002840F092804B4BD3F8E0255D
S31508008EC091B24FF6FF7399420CD0484B03EA8223BE
S31508008ED04FF4F034B4FBF3F403FB04F4C4F5F034B4
S31508008EE0E40A13E04FF48023F2E704F580304FF4E8
S31508008EF0F033B3FBF2F302FB03F34FF4006103EB29
S31508008F00C020FFF72EFF102821D00134364BD3F8A6
S31508008F10E03599B24FF6FF72914220D0334A02EA01
S31508008F2083224FF4F033B3FBF2F302FB03F3C3F5EA
S31508008F30F033DB0A0433A34214D9002DD5D101211D
S31508008F40204600F019FF0028DFD0012040E001216B
S31508008F50204600F011FF0028D7D0012038E04FF452
S31508008F608022DEE700F01AFF1F4BD3F8E02591B206
S31508008F704FF6FF7399422CD01C4B03EA82234FF419
S31508008F80F030B0FBF3F003FB00F0C0F5F03002213F
S31508008F90C00AFFF72DFF20BB154B00221A80124B83
S31508008FA0D3F8E03599B24FF6FF72914214D00F4AC2
S31508008FB002EA83224FF4F033B3FBF2F302FB03F326
S31508008FC0C3F5F033DB0A0B4A13700B4B20221A60E9
S31508008FD038BD4FF48023D2E74FF48022EAE70E200B
S31508008FE0F6E70220F4E700BF0070FF1F00FCFF034E
S31508008FF0E2040020E0040020C000002038B5394B08
S31508009000D3F8E02591B24FF6FF7399420CD0364B50
S3150800901003EA82234FF4F034B4FBF3F403FB04F4BD
S31508009020C4F5F034E40A4CE04FF48023F2E7651CFB
S31508009030A31CAB4207D80221204600F09DFE044639
S31508009040F0B1012449E005F58032D202254BD3F868
S31508009050E01588B24FF6FF7398420ED0224B03EA0A
S3150800906081234FF4F030B0FBF3F003FB0020FFF749
S3150800907091FE042833D10135DAE74FF48023F0E76F
S3150800908000F08CFE29E0184A02EA83224FF4F033F6
S31508009090B3FBF2F302FB03F3C3F5F033DB0A043345
S315080090A0A34219D904F580304FF4F033B3FBF2F339
S315080090B002FB03F303EBC020FFF76CFE0428B6D0CF
S315080090C00234084BD3F8E03599B24FF6FF72914255
S315080090D0D9D14FF48022D9E70524204638BD052486
S315080090E0FBE700BF0070FF1F00FCFF03F8B506464C
S315080090F0614B1D7805F58032D202604BD3F8E01536
S3150800910088B24FF6FF7398424FD05D4B03EA81232E
S315080091104FF4F030B0FBF3F003FB0020FFF73AFE04
S315080091200746564BD3F8E03599B24FF6FF7291428F
S315080091303ED0534A02EA83224FF4F033B3FBF2F3EC
S3150800914002FB03F3C3F5F032A5EBD224013404F095
S31508009150030404EBD22404F5803003EBC020FFF7A8
S3150800916019FE464BD3F8E03599B24FF6FF72914295
S3150800917021D0434A02EA83224FF4F033B3FBF2F3D9
S3150800918002FB03F3C3F5F033A5EBD322033202F057
S31508009190030202EBD322012E10D0022E57D0002E46
S315080091A04CD04FF0FF352846F8BD4FF48023AFE783
S315080091B04FF48022C0E74FF48022DDE7022F19D052
S315080091C0012F4DD12F4B1B68B3F5006FEBD3042845
S315080091D02DD003212846FFF70BFE002843D1012195
S315080091E02046FFF705FE002840D1264B20221A60AC
S315080091F02546D8E7234B1B68B3F5006FD3D304285D
S315080092000ED003212846FFF7F3FD18BB022120469E
S31508009210FFF7EEFD08BB1B4B20221A602546C2E766
S31508009220FFF7ECFE0028ECD04FF0FF35BBE7FFF761
S31508009230E5FE0028CDD04FF0FF35B4E7022FB2D0B7
S31508009240012F02D04FF0FF35ADE71546ABE780B9E1
S315080092502546A8E74FF0FF35A5E74FF0FF35A2E70B
S315080092604FF0FF359FE74FF0FF359CE74FF0FF358E
S3150800927099E74FF0FF3596E7E00400200070FF1FDE
S3150800928000FCFF03C000002082B00B4B9A6C42F42E
S3150800929080529A649B6C03F480530193019B074A9E
S315080092A048F205035361936823F0180343F0080353
S315080092B0936002B0704700BF0010024000300240C1
S315080092C0044B9A6842F001029A601860198018687F
S315080092D080B27047003002402DE9F04780468A4642
S315080092E00020FFF703FFB0F1FF3F63D0814600F58A
S315080092F08035ED02304BD3F8E02591B24FF6FF7377
S3150800930099420CD02D4B03EA82234FF4F032B2FB7C
S31508009310F3F203FB02552846FFF73CFD3EE04FF407
S315080093208023F2E7083C1F2C16D92B19D3E90067CE
S31508009330B7F1FF3F08BFB6F1FF3FF3D0B1B24145E1
S31508009340F0D13846FFF7BCFFB0EB164FEAD1CAF8A2
S3150800935000700020BDE8F087174BD3F8E02591B2DE
S315080093604FF6FF73994220D0144B03EA82234FF439
S31508009370F035B5FBF3F503FB05F5C5F5F033A9EBB9
S31508009380D32909F1030909F0030909EBD32909F5DA
S31508009390803305EBC3252846FFF7FCFC0238C0B22C
S315080093A0022805D84FF4FF64BDE74FF48023DEE7B3
S315080093B00720CFE70320CDE70070FF1F00FCFF035F
S315080093C0431E9BB24FF6FD72934201D9082070479F
S315080093D010B582B00C460023019301A9FFF77CFF64
S315080093E0019B236002B010BD224B1B88B3F5FC7F9E
S315080093F039D270B506460D460120FFF777FEB0F163
S31508009400FF3F32D000F58034E4021B4BD3F8E02549
S3150800941091B24FF6FF73994220D0184B03EA822384
S315080094204FF4F032B2FBF3F203FB024405B9C6B1BE
S3150800943031462846FFF744FF114B196846EA0042B1
S315080094402B46601800F08CFC88B90D4A136808335F
S315080094501360084A13880133138070BD4FF48023C4
S31508009460DEE72846E8E7122070470320F5E70220E2
S31508009470F3E700BFE20400200070FF1F00FCFF03B3
S31508009480C0000020F0B583B005460E4600230193C0
S315080094901746002A4CD10220FFF728FE0446B0F1F1
S315080094A0FF3F00F031819E4B00221A809D4B1870B9
S315080094B09D4B20221A60002F3CD09C4BD3F8E035F8
S315080094C099B24FF6FF7291423BD0994A02EA83223B
S315080094D04FF4F033B3FBF2F302FB03F3C3F5F032B8
S315080094E0A4EBD224033404F0030404EBD22404F5D9
S315080094F0803003EBC020FFF74DFC022824D0042857
S3150800950029D0012F40F00481032840F00381012F60
S3150800951000F0A38031462846FFF766FF002840F092
S31508009520FB807F4B1C88022C40F2E180023CCFE096
S315080095300120B1E70121FFF75BFC0028BDD002231B
S31508009540DFE04FF48022C3E704212046FFF750FCF2
S31508009550002840F0DB80754BD3F8E03599B24FF61A
S31508009560FF72914218D0724A02EA83224FF4F0330E
S31508009570B3FBF2F302FB03F3C3F5F032A4EBD224F8
S31508009580033404F0030404EBD22404F5803003EB1F
S31508009590C020FFF7FFFB20E04FF48022E6E7042116
S315080095A02046FFF725FCF0B10223AAE04FF48022FB
S315080095B04FF4F033B3FBF2F302FB03F3C3F5F032D7
S315080095C0A4EBD224033404F0030404EBD22404F5F8
S315080095D0803003EBC020FFF7DDFBC31EDBB2012B97
S315080095E095D80328DBD0514BD3F8E03599B24FF61E
S315080095F0FF729142DAD04E4A02EA8322D8E74C4AF1
S3150800960002EA81224FF4F031B1FBF2F102FB013399
S315080096100344D3E90023B3F1FF3F08BFB2F1FF3F8C
S315080096201DD03F4A1388013313803F4A1368083315
S3150800963013600830B0F5006F11D23A4B1B7803F56A
S315080096408033DB02394AD2F8E0158CB24FF6FF7246
S315080096509442D4D14FF48022D4E72020EAE7314B54
S315080096601C7800271EE04FF480224FF4F033B3FB3A
S31508009670F2F302FB03F3C3F5F032A4EBD22403346E
S3150800968004F0030404EBD22404F5803003EBC02075
S31508009690FFF780FB03287FF43DAF214A1388FC338C
S315080096A013800137032F3FF635AF204BD3F8E0354B
S315080096B099B24FF6FF729142D5D01D4A02EA83222B
S315080096C0D3E701993046FFF78FFE0346C8B9013440
S315080096D0062C0ED8A542FAD0A6B201A93046FFF745
S315080096E0FBFD03460028ECD00728F0D009E001244A
S315080096F0EEE702210B4B1878FFF77AFB70B94FF4A7
S315080097008073184603B0F0BD0423FAE70223F8E78E
S315080097100A23F6E70A23F4E70223F2E70223F0E72F
S31508009720E2040020E0040020C00000200070FF1FB3
S3150800973000FCFF032DE9F047054600F043FB00282F
S3150800974040F0DD820446FFF79FFDBE4B01221A70EA
S31508009750BD4BD3F8E02591B24FF6FF7399420CD072
S31508009760BA4B03EA82234FF4F037B7FBF3F703FB50
S3150800977007F7C7F5F037FF0A0CE04FF48023F2E746
S315080097801A18B3490A6092ED007B0833B3F5006FE7
S31508009790F6D30137AC4BD3F8E02591B24FF6FF73F9
S315080097A099421AD0A94B03EA82234FF4F036B6FB46
S315080097B0F3F603FB06F6C6F5F036F60A321DBA428C
S315080097C00ED907F580324FF4F030B0FBF3F003FB07
S315080097D000F000EBC2200023D8E74FF48023E4E72B
S315080097E04FF00008974B83F80080C2464746C146AB
S315080097F002E008F101080136934BD3F8E03599B237
S315080098004FF6FF72914228D0904A02EA83224FF41B
S31508009810F033B3FBF2F302FB03F3C3F5F033DB0AD1
S31508009820191DB1421CD906F580304FF4F033B3FB4D
S31508009830F2F302FB03F303EBC020FFF7ABFA431E78
S31508009840DBB2012BD5D90328D5D1B9F1000F00D148
S31508009850B24609F101093746CDE74FF48022D6E72B
S31508009860B8F1000F16D1B9F1000F4CD0AAEB0301DD
S31508009870033101F003010B4403F580334FF4F03054
S31508009880B0FBF2F002FB00F000EBC320FFF782FA10
S31508009890042814D06C4BD3F8E02591B24FF6FF7329
S315080098A0994235D0694B03EA82234FF4F036B6FB6A
S315080098B0F3F603FB06F6C6F5F036F60A42E0624B07
S315080098C0D3F8E03599B24FF6FF72914218D05F4A45
S315080098D002EA83224FF4F033B3FBF2F302FB03F3FD
S315080098E0C3F5F033A7EBD320013000F003000121C4
S315080098F000EBD320FFF77CFA0028CBD00224FFE147
S315080099004FF48022E6E70020FFF7D0FA0446F7E195
S315080099104FF48023C9E74FF4802143E0B31A01339B
S3150800992003F00303134403F580334FF4F030B0FB20
S31508009930F1F001FB00F000EBC320FFF72BFA00283B
S3150800994052D00136404BD3F8E03599B24FF6FF7244
S31508009950914257D03D4A02EA83224FF4F033B3FBD3
S31508009960F2F302FB03F3C3F5F033DB0A0433B34225
S315080099704BD906F580304FF4F033B3FBF2F302FB14
S3150800998003F303EBC020FFF705FA0128D9D12E4BC4
S31508009990D3F8E03599B24FF6FF729142BBD02B4906
S315080099A001EA83214FF4F033B3FBF1F301FB03F330
S315080099B0C3F5F033DA0AB6EBD32FAFD0931CB34214
S315080099C0ACD0B31A033303F00303134403F580330F
S315080099D04FF4F030B0FBF1F001FB00F000EBC320D0
S315080099E0FFF7D8F90328ACD11A4B1E7001220021C3
S315080099F00846FFF747FDB0F5807F40F084814FF0B9
S31508009A00010904E04FF48022A7E74FF000090E4B46
S31508009A10D3F8E02591B24FF6FF7399420ED00B4B5F
S31508009A2003EA82234FF4F036B6FBF3F603FB06F699
S31508009A30C6F5F036F60A4FF0000842E04FF48023E8
S31508009A40F0E700BFD80400200070FF1F00FCFF03EA
S31508009A50DC040020E0040020AF4BD3F8E03599B2CF
S31508009A604FF6FF72914255D0AC4A02EA83224FF470
S31508009A70F033B3FBF2F302FB03F3C3F5F033D90A71
S31508009A80B6EBD32F02D08B1CB34246D1731A0133DF
S31508009A9003F003030B4403F580334FF4F030B0FBB7
S31508009AA0F2F002FB00F000EBC320FFF773F938B9B8
S31508009AB0B8F1000F40F02981994B1E7008F1010892
S31508009AC00136954BD3F8E03599B24FF6FF729142BD
S31508009AD037D0924A02EA83224FF4F033B3FBF2F30B
S31508009AE002FB03F3C3F5F033DB0A191DB1422BD988
S31508009AF006F580304FF4F033B3FBF2F302FB03F3C1
S31508009B0003EBC020FFF746F90228A5D00328D7D1D2
S31508009B103746D5E74FF48022A9E7731A033303F0D3
S31508009B2003030B4403F580334FF4F030B0FBF2F037
S31508009B3002FB00F000EBC320FFF72CF90328BFD186
S31508009B40B6E74FF48022C7E7B8F1000F06D0754B89
S31508009B5000221A802022744B1A602AE0DBB2FA1A15
S31508009B60D2B2013202F003021344D8B26C4B187019
S31508009B700221FFF73DF90028E9D00224C0E04FF49E
S31508009B8080214FF4F030B0FBF1F001FB00331344B1
S31508009B90D3E90001B1F1FF3F08BFB0F1FF3F1CD088
S31508009BA060490B8801330B805F490B6808330B60EB
S31508009BB00832B2F5006F10D2594B1B7803F5803383
S31508009BC0DB025549D1F8E00586B24FF6FF718E42A1
S31508009BD0D5D0524901EA8021D3E7514B1F7827E0B7
S31508009BE04FF480224FF4F033B3FBF2F302FB03F396
S31508009BF0C3F5F033DE0AB7EBD32F25D0B31CBB422F
S31508009C0022D0BF1B033707F00307374407F5803018
S31508009C104FF4F033B3FBF2F302FB03F303EBC0207C
S31508009C20FFF7B8F8032872D13E4A1388FC3313802D
S31508009C30394BD3F8E03599B24FF6FF729142CFD03F
S31508009C40364A02EA8322CDE7354B1B789B1B013344
S31508009C5003F003031E4406F580314FF4F033B3FBDB
S31508009C60F2F302FB03F303EBC12023E04FF4006198
S31508009C70FFF777F8102829D0274BD3F8E03599B2A3
S31508009C804FF6FF72914229D0244A02EA83224FF402
S31508009C90F033B3FBF2F302FB03F3C3F5F032A6EBA2
S31508009CA0D226013606F0030606EBD22606F58032E2
S31508009CB003EBC220B74214D0002DD7D1012130467C
S31508009CC000F05AF80028D7D0012419E001213046BF
S31508009CD000F052F80028CFD0012411E04FF480227A
S31508009CE0D5E700F05BF8B9F1000F09D10021084665
S31508009CF0FFF77AFB68B1122802D0022400E00E248E
S31508009D002046BDE8F0870C24FAE70A24F8E70A2477
S31508009D10F6E70446F4E700BF0070FF1F00FCFF03E8
S31508009D20E0040020E2040020C000002038B5044604
S31508009D300D46FFF759FB122800D038BD00222946E8
S31508009D402046FFF79FFBF8E708B5431E9BB24FF680
S31508009D50FD72934201D9082008BDFFF7E7FFFBE72C
S31508009D6010B5014603484CF2FB3404610020FDF7A8
S31508009D70EFF910BD0020024000B587B0002301931B
S31508009D800293059104900123039301A902A8FDF704
S31508009D908DFA00B1012007B05DF804FB084B1A687C
S31508009DA022F480621A601A6842F480521A601A68AD
S31508009DB022F480521A601A6842F480621A60704768
S31508009DC0002002400020704708B502F042FB10B19F
S31508009DD002684068904708BDEFF305832BB9064B28
S31508009DE0186828B901221A6070476FF00500704795
S31508009DF04FF0FF30704700BF340C0020EFF30583A7
S31508009E0073B90A4B1B68012B0DD110B50024084BFA
S31508009E10DC77064B02221A6001F0EEFB204610BDE5
S31508009E206FF0050070474FF0FF307047340C002084
S31508009E3000ED00E008B5EFF3058343B901F066FFCE
S31508009E4040B1022808D101F02DFC002008BD6FF0B2
S31508009E500500FBE70120F9E74FF0FF30F6E7F0B51C
S31508009E6087B000240594EFF3058404BBF8B1002AF3
S31508009E7034D0156893692BB11E46013B372B02D99E
S31508009E80002015E01826536813F0010F3FD15469D6
S31508009E9084B14FEA940C93682BB1D768A72F02D9DF
S31508009EA0176907B184B943B14FF0FF330BB305986F
S31508009EB007B0F0BD4FF0800CEDE7D368A3B913697E
S31508009EC0ABB14FF0FF33F1E70293019700960B46CB
S31508009ED06246294601F022FB0590E8E7154600236D
S31508009EE018264FF0800CE1E74FF0FF33DEE700233A
S31508009EF0DCE705AB019300960B461FFA8CF2294660
S31508009F0001F047FB0128D2D000230593CFE70020B4
S31508009F10CEE708B5EFF3058323B930B101F050FD5C
S31508009F20002008BD6FF00500FBE76FF00300F8E7B7
S31508009F3008B5EFF3058333B908B9002008BD01F069
S31508009F40C7FC0020FAE76FF00500F7E72DE9F043B4
S31508009F5083B0EFF30587002F43D106468946154699
S31508009F601C4600283FD0082002F0BCFC804600288A
S31508009F703BD006604560B9F1000F00D0012704B355
S31508009F802068A36813B1E2682B2A10D853B14FF0A2
S31508009F90FF33DBB10024404602F026FD204603B01D
S31508009FA0BDE8F083E3687BB14FF0FF33F1E7019337
S31508009FB00F4B009343463A46012102F095F80446B2
S31508009FC00CE020460023E4E70023E2E7084B009371
S31508009FD043463A46012102F06BF80446002CDDD1CF
S31508009FE0D9E70024DAE70024D8E70446D6E700BF15
S31508009FF0C99D0008EFF305836BB90A4670B100B531
S3150800A00083B00093042102F099F8012809D10020B1
S3150800A01003B05DF804FB6FF0050070476FF00300AE
S3150800A02070476FF00200F3E708B5EFF30583CBB985
S3150800A030A0B1836813B1C2681F2A0BD82BB14FF0A1
S3150800A040FF338BB900F052FA08BDC36843B14FF02D
S3150800A050FF33F6E7184600F024FAF5E70023F0E7A1
S3150800A0600023EEE70020EFE70020EDE7F8B110B592
S3150800A07082B00C46B1F1807F1CD2EFF305829AB10B
S3150800A0800022019201AA00F04FFBB8B1019BC3B1AF
S3150800A0904FF0E0234FF08052C3F8042DBFF34F8FE3
S3150800A0A0BFF36F8F204607E000F0F2FA04E06FF086
S3150800A0B0030070476FF0030002B010BD6FF0020096
S3150800A0C0FAE72046F8E770B5B0B10C460646B1F196
S3150800A0D0807F14D2EFF3058353B100F0CBFA05461F
S3150800A0E02146304600F0BCFA58B96FF0020508E080
S3150800A0F000F08FFA054604E06FF0030501E06FF003
S3150800A1000305284670BD40B370B582B00C461D469F
S3150800A1108446B1F1807F23D2EFF3058323BB12F087
S3150800A120010610D0012312F0020F0ED0002200956E
S3150800A1302146604600F0E8F94EB1844312D0B5B125
S3150800A1406FF001000EE00023EDE70122EFE704427D
S3150800A15008D17DB16FF0010004E06FF0030070478D
S3150800A1606FF0030002B070BD6FF00500FAE76FF0FC
S3150800A1700200F7E76FF00200F4E770B5EFF3058623
S3150800A180002E3ED1044608B3436813F0010600D0FA
S3150800A190012613F0080F37D154B3A16811B1E3684B
S3150800A1A04F2B1AD8A1B14FF0FF337BBB26B304203F
S3150800A1B000F042FD05462DB304B124682146284621
S3150800A1C000F0D4FFF6B145F001051BE03346E0E7A1
S3150800A1D0E3687BB14FF0FF33E7E726B1042000F0D0
S3150800A1E036FD0546E7E7012000F031FD0546E2E7C2
S3150800A1F00023DAE70023D8E7012000F01DFD054615
S3150800A200D9E70025284670BD0025FBE70025F9E7B4
S3150800A210EFF30582DAB910B503460C4620F00100C3
S3150800A22003F00101012B15D941B1214600F027FFA2
S3150800A230012812D09CB16FF001000FE0214600F012
S3150800A2404BFE01280ED07CB16FF0010006E06FF0DE
S3150800A250050070476FF0030000E0002010BD6FF0A6
S3150800A2600200FBE70020F9E76FF00200F6E7EFF3DC
S3150800A2700582BAB908B5034620F0010003F00101CA
S3150800A280012B12D929B100F0F1FC012810D10020C8
S3150800A29008BD00231A46194600F0FEFB01280AD11C
S3150800A2A00020F5E76FF0050070476FF00300EFE751
S3150800A2B06FF00200ECE76FF00200E9E770B582B0D4
S3150800A2C0EFF30583002B3AD1144600283BD000292A
S3150800A2D03BD06AB393684BB1D2684F2A06D9226934
S3150800A2E022B101FB00F56669AE421BD273B14FF08D
S3150800A2F0FF3363BB002200F0ABFB054605B304B190
S3150800A30024682146284600F031FF19E0E3688BB936
S3150800A310236913B14FF0FF33EBE763696BB14FF075
S3150800A320FF33E6E70025009500F048FB0546E5E71C
S3150800A3300023DEE74FF0FF33DBE70023D9E70025EC
S3150800A340284602B070BD0025FAE70025F8E7002583
S3150800A350F6E710B582B01C46EFF30583C3B118B310
S3150800A36029B33CBB0023019301AA00F09FFC0128F6
S3150800A37023D1019850B14FF0E0234FF08052C3F833
S3150800A380042DBFF34F8FBFF36F8F002002B010BDAF
S3150800A390B0B1C1B10023224600F07EFB012815D0DA
S3150800A3A0B4B16FF00100F1E76FF00300EEE76FF06C
S3150800A3B00300EBE76FF00300E8E76FF00200E5E75C
S3150800A3C06FF00300E2E76FF00300DFE70020DDE748
S3150800A3D06FF00200DAE710B582B01C46EFF305838A
S3150800A3E0C3B110B321B334BB0023019301AA00F013
S3150800A3F066FE012822D1019850B14FF0E0234FF0B4
S3150800A4008052C3F8042DBFF34F8FBFF36F8F002020
S3150800A41002B010BDA8B1B9B1224600F0AEFC0128C1
S3150800A42015D0B4B16FF00100F2E76FF00300EFE763
S3150800A4306FF00300ECE76FF00300E9E76FF0020046
S3150800A440E6E76FF00300E3E76FF00300E0E70020BC
S3150800A450DEE76FF00200DBE7034B0360034B0B609C
S3150800A46080231360704700BF8C0B00208C090020E6
S3150800A470034B0360034B0B604FF480731360704704
S3150800A480E4080020E40400201AB9084205D1104661
S3150800A4907047814303D00020704701207047012090
S3150800A4A0704780B110B582B0044620230193019B02
S3150800A4B0202B11D04FF0500383F31188BFF36F8F11
S3150800A4C0BFF34F8FFEE74FF0500383F31188BFF3B6
S3150800A4D06F8FBFF34F8FFEE7002340F8043B00F071
S3150800A4E02DF901232377204602B010BD38B5202068
S3150800A4F002F0F8F9044628B1002540F8045B00F09C
S3150800A5001DF92577204638BD88B12DE9F0410C465E
S3150800A51016461D460746B1F1807F11D34FF050030A
S3150800A52083F31188BFF36F8FBFF34F8FFEE74FF0AA
S3150800A530500383F31188BFF36F8FBFF34F8FFEE786
S3150800A54041B94FF0500383F31188BFF36F8FBFF300
S3150800A5504F8FFEE701F0DAFB50B9069B43B14FF087
S3150800A560500383F31188BFF36F8FBFF34F8FFEE756
S3150800A57001F098F8D7F800802A4621464046FFF7AA
S3150800A58083FFF8B18EB328EA04033B6000230693E1
S3150800A59001F022F9069B93B148B94FF0E0234FF03A
S3150800A5A08052C3F8042DBFF34F8FBFF36F8F01F0AE
S3150800A5B0A1FC804610F0007F1AD028F07F4840465C
S3150800A5C0BDE8F081069B002BE2D05EB900210DB1F3
S3150800A5D041F08061069A2143381D01F06BFA4FF06D
S3150800A5E00008D5E74FF08071F1E700230693CFE71F
S3150800A5F001F0C0FFD7F800802A4621464046FFF7FB
S3150800A60043FF18B116B128EA04043C6001F0D4FFF0
S3150800A610D3E770B170B50C460546B1F1807F11D30A
S3150800A6204FF0500383F31188BFF36F8FBFF34F8F3B
S3150800A630FEE74FF0500383F31188BFF36F8FBFF324
S3150800A6404F8FFEE701F096FF2E6826EA04042C6079
S3150800A65001F0B2FF304670BD08B5FFF7DAFF08BD56
S3150800A66008B50A4600230146014801F005FF08BD62
S3150800A67059A60008EFF311834FF0500282F31188B0
S3150800A680BFF36F8FBFF34F8F006883F3118870474E
S3150800A690F8B568B10D460446B1F1807F11D34FF085
S3150800A6A0500383F31188BFF36F8FBFF34F8FFEE715
S3150800A6B04FF0500383F31188BFF36F8FBFF34F8FAB
S3150800A6C0FEE700F10C0600F0EDFF206923682B4336
S3150800A6D0236000270AE0216832EA010105D111E06A
S3150800A6E0216841F0007101F073FA2846B0420ED095
S3150800A6F04568036823F07F4213F0806FEBD1216829
S3150800A7001142F2D013F0807FEAD01743E8E72368B6
S3150800A71023EA0703236001F05FF82068F8BD08B54F
S3150800A720FFF7B6FF08BD000008B513460A460146FE
S3150800A730014801F0A1FE08BD1FA7000800F10803A3
S3150800A74043604FF0FF328260C360036100230360F9
S3150800A750704700230361704743684B609A688A60B4
S3150800A760516099600861036801330360704730B42B
S3150800A7700D68B5F1FF3F11D000F108031C465B6870
S3150800A7801A68AA42FAD963684B6099608C6061605E
S3150800A790086103680133036030BC70470469F2E757
S3150800A7A00369416882688A60416851605A688242D2
S3150800A7B006D0002202611A68013A1A6018687047C2
S3150800A7C082685A60F5E70346406A18B11B6B186839
S3150800A7D0C0F13800704710B5044601F0CBFEA26BF5
S3150800A7E0E36B9A4204D0002401F0E6FE204610BD31
S3150800A7F00124F9E710B5044601F0BCFEA36B23B9A2
S3150800A800012401F0D9FE204610BD0024F9E770B5F1
S3150800A81004461546866B026C5AB903681BB10020BC
S3150800A8200136A66370BD806801F0CCFA0023A360E8
S3150800A830F6E76DB9406802F0CBF96368226C1344F9
S3150800A8406360A268934219D3236863602846E7E7E2
S3150800A850C06802F0BDF9E368226C51429B1AE360B6
S3150800A8602268934202D2A3680B44E360022D01D00A
S3150800A8700020D5E726B1013E0020D1E72846CFE7DC
S3150800A8800020CDE70346026C6AB110B50846D968C0
S3150800A8901144D9609C68A14201D31968D960D96866
S3150800A8A002F096F910BD704738B5054601F062FE0C
S3150800A8B095F8454064B201E0013C64B2002C0ADD1B
S3150800A8C06B6A43B105F1240001F03CF90028F3D086
S3150800A8D001F010FAF0E7FF2385F8453001F06CFE29
S3150800A8E001F048FE95F8444064B201E0013C64B2C8
S3150800A8F0002C0ADD2B6943B105F1100001F022F99D
S3150800A9000028F3D001F0F6F9F0E7FF2385F8443084
S3150800A91001F052FE38BD38B5E0B10D46044601F0E7
S3150800A92029FE2368E26B216C01FB0230A06000203F
S3150800A930A0636360013A02FB0133E360FF2384F8F6
S3150800A940443084F84530FDB9236963B901F034FE13
S3150800A950012038BD4FF0500383F31188BFF36F8F82
S3150800A960BFF34F8FFEE704F1100001F0EBF8002863
S3150800A970ECD04FF0E0234FF08052C3F8042DBFF31C
S3150800A9804F8FBFF36F8FE1E704F11000FFF7D6FE94
S3150800A99004F12400FFF7D2FED8E738B51D46049C1B
S3150800A9A00B4649B92460E063236401212046FFF77A
S3150800A9B0B2FF84F84C5038BD2260F4E740B94FF036
S3150800A9C0500383F31188BFF36F8FBFF34F8FFEE7F2
S3150800A9D010B584B01C46844653B192B189B94FF07C
S3150800A9E0500383F31188BFF36F8FBFF34F8FFEE7D2
S3150800A9F04FF0500383F31188BFF36F8FBFF34F8F68
S3150800AA00FEE76AB150230393039B502B13D04FF0F4
S3150800AA10500383F31188BFF36F8FBFF34F8FFEE7A1
S3150800AA200029EFD04FF0500383F31188BFF36F8FDF
S3150800AA30BFF34F8FFEE7039B012384F8463000944B
S3150800AA409DF818306046FFF7A8FF204604B010BDF1
S3150800AA5040B94FF0500383F31188BFF36F8FBFF3EC
S3150800AA604F8FFEE7F0B583B00D461446064601FB48
S3150800AA7000F0503001F036FF074650B1002380F849
S3150800AA8046300090234600F1500229463046FFF72B
S3150800AA9084FF384603B0F0BDF0B585B0019288B1A1
S3150800AAA00F461D460446B1B1022D20D1E36B012B9A
S3150800AAB01DD04FF0500383F31188BFF36F8FBFF398
S3150800AAC04F8FFEE74FF0500383F31188BFF36F8F64
S3150800AAD0BFF34F8FFEE7036C002BE5D04FF0500312
S3150800AAE083F31188BFF36F8FBFF34F8FFEE701F033
S3150800AAF00DF9064658B9019B002B48D04FF0500374
S3150800AB0083F31188BFF36F8FBFF34F8FFEE70026DD
S3150800AB103DE02A4639462046FFF779FE636A7BB947
S3150800AB2048B14FF0E0234FF08052C3F8042DBFF32D
S3150800AB304F8FBFF36F8F01F03FFD012005B0F0BDC9
S3150800AB4004F1240000F0FEFF0028F4D04FF0E023C3
S3150800AB504FF08052C3F8042DBFF34F8FBFF36F8FAA
S3150800AB60E9E701F029FD0020E8E702A801F074F8FA
S3150800AB70012619E0002384F8443021E0002384F8F4
S3150800AB80453023E02046FFF78FFE00F025FE01F052
S3150800AB90F1FCA26BE36B9A42BBD3022DB9D0019BA1
S3150800ABA0002BDED0002EE0D001F006FD00F07AFD85
S3150800ABB001F0E0FC94F8442052B2B2F1FF3FD9D03C
S3150800ABC094F8452052B2B2F1FF3FD7D001F0F4FC19
S3150800ABD001A902A801F04CF8D8B92046FFF7FBFDF9
S3150800ABE00028CFD0019904F1100000F04BFF204651
S3150800ABF0FFF75AFE00F0F0FD0028C8D14FF0E02319
S3150800AC004FF08052C3F8042DBFF34F8FBFF36F8FF9
S3150800AC10BDE72046FFF748FE00F0DEFD00208DE781
S3150800AC2048B108B5002181600160C1600B460A463B
S3150800AC30FFF732FF08BD704710B502460021012014
S3150800AC40FFF706FF0446FFF7EBFF204610BD10B5D9
S3150800AC5082B00B460090002211460120FFF7AEFE97
S3150800AC600446FFF7DDFF204602B010BD38B538B1FF
S3150800AC700446856801F044F885420AD0002038BDAC
S3150800AC804FF0500383F31188BFF36F8FBFF34F8FD5
S3150800AC90FEE7E368013BE3600BB10120EFE71A46E4
S3150800ACA019462046FFF7F8FE0120E8E72DE9F843A4
S3150800ACB090B10F4616461C460546B1B1022C20D166
S3150800ACC0EB6B012B1DD04FF0500383F31188BFF3B4
S3150800ACD06F8FBFF34F8FFEE74FF0500383F3118852
S3150800ACE0BFF36F8FBFF34F8FFEE7036C002BE5D0E2
S3150800ACF04FF0500383F31188BFF36F8FBFF34F8F65
S3150800AD00FEE701F05DFDEFF311884FF0500383F382
S3150800AD101188BFF36F8FBFF34F8FAA6BEB6B9A4205
S3150800AD2006D3022C04D0002088F31188BDE8F883E6
S3150800AD3095F845904FFA89F9AB6B2246394628466D
S3150800AD40FFF765FDB9F1FF3F06D009F101035BB2D4
S3150800AD5085F845300120E7E76B6A0BB90120E3E780
S3150800AD6005F1240000F0EEFE18B126B1012030608E
S3150800AD70DAE70120D8E70120D6E7F0B585B00192D9
S3150800AD8090B10F460446C1B100F0C0FF064600BBAD
S3150800AD90019B002B5ED04FF0500383F31188BFF35D
S3150800ADA06F8FBFF34F8FFEE74FF0500383F3118881
S3150800ADB0BFF36F8FBFF34F8FFEE7036C002BE3D013
S3150800ADC04FF0500383F31188BFF36F8FBFF34F8F94
S3150800ADD0FEE700263EE039462046FFF753FD013DD3
S3150800ADE0A563236923B901F0E7FB012005B0F0BD8F
S3150800ADF004F1100000F0A6FE0028F4D04FF0E0237E
S3150800AE004FF08052C3F8042DBFF34F8FBFF36F8FF7
S3150800AE10E9E701F0D1FB0020E8E702A800F01CFFF3
S3150800AE20012621E0002384F8443029E0002384F831
S3150800AE3045302BE02046FFF737FD00F0CDFC09E052
S3150800AE402046FFF731FD00F0C7FC2046FFF7D2FC8D
S3150800AE5000283FD101F08EFBA56B002DBBD1019BCD
S3150800AE60002BD6D0002ED8D001F0A6FB00F01AFC95
S3150800AE7001F080FB94F844305BB2B3F1FF3FD1D0C8
S3150800AE8094F845305BB2B3F1FF3FCFD001F094FBA5
S3150800AE9001A902A800F0ECFE0028D1D12046FFF750
S3150800AEA0A9FC0028C6D0019904F1240000F0EAFDA7
S3150800AEB02046FFF7F9FC00F08FFC0028CAD14FF0B6
S3150800AEC0E0234FF08052C3F8042DBFF34F8FBFF332
S3150800AED06F8FBFE7002089E770B584B0019158B13C
S3150800AEE00446036C8BB14FF0500383F31188BFF30C
S3150800AEF06F8FBFF34F8FFEE74FF0500383F3118830
S3150800AF00BFF36F8FBFF34F8FFEE700F0FFFE0546D6
S3150800AF1050B9019B5BB14FF0500383F31188BFF31F
S3150800AF206F8FBFF34F8FFEE70026354655E006467E
S3150800AF3053E0013BA36323683BB123694BB901F096
S3150800AF403BFB0126304604B070BD00F0DFFFA06071
S3150800AF50F3E704F1100000F0F5FD0028EFD04FF0FC
S3150800AF60E0234FF08052C3F8042DBFF34F8FBFF391
S3150800AF706F8FE4E746B14FF0500383F31188BFF3B0
S3150800AF806F8FBFF34F8FFEE701F016FBDAE702A8D3
S3150800AF9000F062FE01252AE0002384F8443032E0FE
S3150800AFA0002384F8453034E001F0E4FAA06800F0A4
S3150800AFB0BDFE064601F000FB3BE02046FFF774FCA9
S3150800AFC000F00AFC09E02046FFF76EFC00F004FCDE
S3150800AFD02046FFF70FFC002842D101F0CBFAA36BFD
S3150800AFE0002BA6D1019B002BC4D0002DCFD001F099
S3150800AFF0E3FA00F057FB01F0BDFA94F844305BB26F
S3150800B000B3F1FF3FC8D094F845305BB2B3F1FF3FC8
S3150800B010C6D001F0D1FA01A902A800F029FE00283D
S3150800B020D1D12046FFF7E6FB0028C6D02368002BBF
S3150800B030BAD0019904F1240000F024FD2046FFF758
S3150800B04033FC00F0C9FB0028C7D14FF0E0234FF0CE
S3150800B0508052C3F8042DBFF34F8FBFF36F8FBCE741
S3150800B0600EB900266EE701F085FA2046FFF7ABFB1E
S3150800B0700146A06800F0EEFE01F09EFAF1E780B105
S3150800B08070B50C460546866800F03AFE864211D031
S3150800B09021462846FFF720FF80B1EB680133EB60B5
S3150800B0A00CE04FF0500383F31188BFF36F8FBFF3A3
S3150800B0B04F8FFEE7EB680133EB60012070BD2DE989
S3150800B0C0F843B0B10D4690460446D9B101F078FB75
S3150800B0D0EFF311874FF0500383F31188BFF36F8F97
S3150800B0E0BFF34F8FA66BCEB9002087F31188BDE852
S3150800B0F0F8834FF0500383F31188BFF36F8FBFF3C4
S3150800B1004F8FFEE7036C002BE0D04FF0500383F31C
S3150800B1101188BFF36F8FBFF34F8FFEE794F8449003
S3150800B1204FFA89F929462046FFF7ACFB731EA3633D
S3150800B130B9F1FF3F06D009F101035BB284F8443048
S3150800B1400120D2E723690BB90120CEE704F11000EC
S3150800B15000F0F8FC30B1B8F1000F05D00120C8F8AE
S3150800B1600000C2E70120C0E70120BEE70023072B45
S3150800B1700CD8074A52F833200AB10133F7E7044AD4
S3150800B18042F8331002EBC30250607047704700BFA5
S3150800B190380C002070B504460D46164601F0EAF94B
S3150800B1A094F844305BB2B3F1FF3F0DD094F84530C4
S3150800B1B05BB2B3F1FF3F0BD001F0FEF9A36B5BB1B5
S3150800B1C02046FFF771FB70BD002384F84430EDE795
S3150800B1D0002384F84530EFE73246294604F1240077
S3150800B1E000F094FCECE70000084B1B681B6823B9C9
S3150800B1F0074B4FF0FF321A607047044B1B68DB6839
S3150800B200DB685A68024B1A60704700BFE80C0020DA
S3150800B210800C00202DE9F04780460D4617469946D2
S3150800B220089EDDF824A00A9C9200A521206B01F057
S3150800B23042FC236B07F18042013A03EB820727F0B1
S3150800B2400707002D42D04FF0000CBCF10F0F09D8AC
S3150800B25015F80C3004EB0C0282F8343013B10CF1FB
S3150800B260010CF2E7002384F84330372E00D937263D
S3150800B270E662E66400252565201DFFF76AFA04F1F3
S3150800B2801800FFF766FA2461C6F13806A6616462FB
S3150800B290C4F8A05084F8A4504C22294604F154005E
S3150800B2A001F009FC0B4BA36503F16802E265D03394
S3150800B2B023664A464146384601F030F92060BAF11D
S3150800B2C0000F01D0CAF80040BDE8F087002384F8D3
S3150800B2D03430CAE7CC92002038B5002407E004EBE6
S3150800B2E0840293000E481844FFF728FA0134372CD5
S3150800B2F0F5D90C4D2846FFF721FA0B4C2046FFF7E7
S3150800B3001DFA0A48FFF71AFA0948FFF717FA094813
S3150800B310FFF714FA084B1D60084B1C6038BD00BFC8
S3150800B320140D0020000D0020EC0C0020D00C00208D
S3150800B330BC0C0020A40C0020E80C0020E40C002023
S3150800B34010B5044601F016F9224A13680133136052
S3150800B350214B1B685BB1214B1B686BB91E4B1B68E5
S3150800B360DA6AE36A9A4207D81B4B1C6004E01A4B58
S3150800B3701C601368012B29D0194A1368013313601E
S3150800B3806364E06A174B1B68984201D9154B18602D
S3150800B39000EB8000211D144B03EB8000FFF7DCF95E
S3150800B3A001F00AF90D4B1B687BB10B4B1B68DA6A77
S3150800B3B0E36A9A4209D24FF0E0234FF08052C3F86D
S3150800B3C0042DBFF34F8FBFF36F8F10BDFFF784FFB8
S3150800B3D0D2E700BFA00C002074110020940C0020B6
S3150800B3E0840C0020980C0020140D002010B504468B
S3150800B3F0543001F069FB94F8A53063B1012B11D0E4
S3150800B400022B0ED04FF0500383F31188BFF36F8FD2
S3150800B410BFF34F8FFEE7206B01F0E6FA204601F0F6
S3150800B420E3FA10BD204601F0DFFAFAE70F4B1B6876
S3150800B430D3B110B501F09EF80D4BDB68DC68201D12
S3150800B440FFF7AEF90B4A1368013B1360074A136806
S3150800B450013B136001F0B0F82046FFF7C7FF034B26
S3150800B4601B68002BE6D110BD704700BFB80C002042
S3150800B470BC0C0020A00C002008B5FFF7D7FF074B2F
S3150800B4801B68012BF9D94FF0E0234FF08052C3F81F
S3150800B490042DBFF34F8FBFF36F8FEEE7140D002017
S3150800B4A070B504460D46174B1E68174B18680430CE
S3150800B4B0FFF776F9B4F1FF3F0DD03444124B1B6801
S3150800B4C05C60A64210D9114B18680F4B19680431F5
S3150800B4D0FFF74DF970BD002DEFD00B4B19680431FD
S3150800B4E00B48FFF739F9F5E70A4B1868064B196850
S3150800B4F00431FFF73CF9084B1B68A342EAD9064B0F
S3150800B5001C60E7E79C0C002074110020E40C002066
S3150800B510A40C0020E80C0020800C002030B587B071
S3150800B5200B9C7CB10C9DB5B1A8250495049DA82D4E
S3150800B5301AD04FF0500383F31188BFF36F8FBFF310
S3150800B5404F8FFEE74FF0500383F31188BFF36F8FD9
S3150800B550BFF34F8FFEE74FF0500383F31188BFF315
S3150800B5606F8FBFF34F8FFEE7049D0C9D2C6302245B
S3150800B57085F8A54000240394029505AC01940A9C1D
S3150800B5800094FFF747FE0C98FFF7DAFE059807B018
S3150800B59030BD2DE9F04385B00746884614461E4659
S3150800B5A0900001F09FF908B38146A82001F09AF9A6
S3150800B5B00546A8B1C0F83090002380F8A53003935B
S3150800B5C002900D9B01930C9B0093334622464146FD
S3150800B5D03846FFF71FFE2846FFF7B2FE012007E0B0
S3150800B5E0484601F001FA4FF0FF3001E04FF0FF3016
S3150800B5F005B0BDE8F083000010B588B000240594B6
S3150800B600069407AA06A905A8FEF726FF059B029336
S3150800B610069B019300942346079A1A491A48FFF78E
S3150800B6207DFF1A4B1860E8B100F010FD01281AD109
S3150800B6304FF0500383F31188BFF36F8FBFF34F8F1B
S3150800B640134B1B685433134A1360134B4FF0FF32E6
S3150800B6501A60124B01221A60114B00221A6001F07F
S3150800B66023F803E00020B0F1FF3F01D008B010BD79
S3150800B6704FF0500383F31188BFF36F8FBFF34F8FDB
S3150800B680FEE700BF04CE000879B400087C0C002051
S3150800B69074110020C8000020800C0020940C0020A3
S3150800B6A09C0C0020024A136801331360704700BFE0
S3150800B6B0780C0020014B1868704700BF9C0C0020CE
S3150800B6C0F8B53A4B1B68002B69D1394B1D68013513
S3150800B6D01D60C5B9374B1B681B6843B14FF0500353
S3150800B6E083F31188BFF36F8FBFF34F8FFEE7314A9D
S3150800B6F01168314B186810601960304A13680133B5
S3150800B7001360FFF771FD2E4B1B68AB423DD900272E
S3150800B7102C4B1B68DB6A03EB83039A002A4B9B5866
S3150800B720012B00D90127294B1B68002B3CD0012788
S3150800B7303AE001271F4B1B681B6843B31D4B1B6868
S3150800B740DB68DC6863689D4226D3261D3046FFF712
S3150800B75027F8A36A1BB104F11800FFF721F8E36A7A
S3150800B7601B4A1268934201D9194A136003EB8303F3
S3150800B7709A00314614481044FEF7EEFFE26A114B70
S3150800B7801B68DB6A9A42D4D2D4E70027D2E70C4B6F
S3150800B7904FF0FF321A60BBE7094A1360B8E70D4A53
S3150800B7A013680133136000273846F8BD780C00206B
S3150800B7B09C0C0020E80C0020E40C0020880C0020DB
S3150800B7C0800C002074110020140D00208C0C002021
S3150800B7D0980C0020900C002038B5354B1B6843B9EF
S3150800B7E04FF0500383F31188BFF36F8FBFF34F8F6A
S3150800B7F0FEE700F0BFFE2E4B1A68013A1A601B6876
S3150800B800002B4FD12B4B1B680BB900244BE00024AF
S3150800B810294B1B681BB3284BDB68DC6804F118004E
S3150800B820FEF7BEFF251D2846FEF7BAFFE06A234B42
S3150800B8301B68984201D9214B186000EB8000294605
S3150800B8401F4B03EB8000FEF787FFE26A1D4B1B6860
S3150800B850DB6A9A42DCD31C4B01221A60D8E70CB18A
S3150800B860FFF7C2FC194B1C6884B9174B1C68D4B186
S3150800B8704FF0E0234FF08052C3F8042DBFF34F8FEB
S3150800B880BFF36F8F01240EE0013C07D0FFF718FFC6
S3150800B8900028F9D00C4B01221A60F5E70B4B002261
S3150800B8A01A60E2E7002400F087FE204638BD00BF94
S3150800B8B0780C0020A00C0020D00C0020980C00204A
S3150800B8C0140D0020741100208C0C0020900C002010
S3150800B8D010B5A8B10446104B1B6843B14FF050038E
S3150800B8E083F31188BFF36F8FBFF34F8FFEE7FFF720
S3150800B8F0D9FE00212046FFF7D3FDFFF76DFF48B9B3
S3150800B9004FF0E0234FF08052C3F8042DBFF34F8F5A
S3150800B910BFF36F8F10BD00BF780C0020224B1B6849
S3150800B9201BB1224B01221A607047204B00221A6075
S3150800B9301F4B1B6803EB83018A001E498A585AB9B4
S3150800B9400BB1013BF6E74FF0500383F31188BFF3C1
S3150800B9506F8FBFF34F8FFEE7084603EB83018A001C
S3150800B960024451684968516003EB830C4FEA8C0224
S3150800B9700832024491420FD003EB830291000D4A2C
S3150800B9800A445268D1680C4A116009490B60136869
S3150800B99054330A4A13607047486862469100054A5C
S3150800B9A00A445060E8E700BF780C00208C0C0020A1
S3150800B9B0980C0020140D002074110020C8000020E7
S3150800B9C038B5044600F0D6FDE4B1251D2846FEF735
S3150800B9D0E7FEA36A1BB104F11800FEF7E1FE29464B
S3150800B9E02348FEF7B9FE94F8A430DBB2012B0CD03D
S3150800B9F000F0E2FD1F4B1B685BB91F4B1B68A34297
S3150800BA000ED038BD1C4B1C68DFE7002384F8A43031
S3150800BA10EEE700F0AFFDFFF7E7FB00F0CDFDECE742
S3150800BA20144B1B68B3B1154B1B6843B14FF0500359
S3150800BA3083F31188BFF36F8FBFF34F8FFEE74FF085
S3150800BA40E0234FF08052C3F8042DBFF34F8FBFF3A6
S3150800BA506F8FD6E7064B1A68094B1B689A4203D1C3
S3150800BA60054B00221A60CCE7FFF758FFC9E700BF6D
S3150800BA70A40C0020940C002074110020780C0020DF
S3150800BA80A00C002058B110B50C46094A11681831A7
S3150800BA90FEF76DFE01212046FFF702FD10BD4FF0AF
S3150800BAA0500383F31188BFF36F8FBFF34F8FFEE701
S3150800BAB07411002070B110B514460246114B1B686C
S3150800BAC08BB94FF0500383F31188BFF36F8FBFF321
S3150800BAD04F8FFEE74FF0500383F31188BFF36F8F44
S3150800BAE0BFF34F8FFEE7084B186841F000418161AC
S3150800BAF0196818311046FEF72FFE01212046FFF778
S3150800BB00CFFC10BD780C00207411002038B570B138
S3150800BB100D4614460A4A11681831FEF71DFE0CB187
S3150800BB204FF0FF3521462846FFF7BAFC38BD4FF0DF
S3150800BB30500383F31188BFF36F8FBFF34F8FFEE770
S3150800BB407411002038B5C368DC6824B304F11805FD
S3150800BB502846FEF725FE184B1B682BBB251D2846D5
S3150800BB60FEF71EFEE06A154B1B68984201D9134B77
S3150800BB70186000EB80002946114B03EB8000FEF7A6
S3150800BB80EBFDE26A0F4B1B68DB6A9A4211D901206A
S3150800BB900D4B186038BD4FF0500383F31188BFF37F
S3150800BBA06F8FBFF34F8FFEE729460848FEF7D4FD8F
S3150800BBB0E7E70020EEE700BF780C0020980C00208D
S3150800BBC0140D0020741100208C0C0020D00C0020CD
S3150800BBD038B51C4B1B6843B94FF0500383F31188E3
S3150800BBE0BFF36F8FBFF34F8FFEE741F0004101604F
S3150800BBF0C468F4B1FEF7D4FD251D2846FEF7D0FD2E
S3150800BC00E06A114B1B68984201D90F4B186000EB8C
S3150800BC10800029460D4B03EB8000FEF79DFDE26A86
S3150800BC200B4B1B68DB6A9A4202D90A4B01221A603F
S3150800BC3038BD4FF0500383F31188BFF36F8FBFF3FE
S3150800BC404F8FFEE7780C0020980C0020140D00207A
S3150800BC50741100208C0C0020034B1B680360034BF7
S3150800BC601B684360704700BF880C00209C0C0020AE
S3150800BC70F8B5C8B10C460546F9B100F07BFC1B4B7C
S3150800BC8019686B68C81A2268B2F1FF3F26D0184EA9
S3150800BC9036682F68B74201D08B4224D9824215D81C
S3150800BCA00023236001241AE04FF0500383F3118820
S3150800BCB0BFF36F8FBFF34F8FFEE74FF0500383F349
S3150800BCC01188BFF36F8FBFF34F8FFEE75B1A1344DC
S3150800BCD023602846FFF7C0FF002400E0002400F098
S3150800BCE06BFC2046F8BD0124F9E700BF9C0C002038
S3150800BCF0880C0020014B01221A6070478C0C00202A
S3150800BD00014B1868704700BF74110020054B1B686B
S3150800BD1033B1054B1B680BB10020704702207047F2
S3150800BD2001207047940C0020780C002000283ED093
S3150800BD3038B50446C36A204A1268D26A93422ED29C
S3150800BD408269002A05DB1C4A1268D26AC2F13802E7
S3150800BD508261616903EB8303184A02EB8303994204
S3150800BD6005D0154B1B68DB6AE362012038BD251D2B
S3150800BD702846FEF715FD104B1B68D86AE062104B83
S3150800BD801B68984201D90E4B186000EB80002946C3
S3150800BD900A4B03EB8000FEF7DFFC0120E6E7C26CE6
S3150800BDA0054B1B68DB6A9A4203D30020DEE70020B6
S3150800BDB070470120DAE700BF74110020140D002037
S3150800BDC0980C002000283BD038B504461E4B1B684B
S3150800BDD0834208D04FF0500383F31188BFF36F8F67
S3150800BDE0BFF34F8FFEE7036D43B94FF0500383F35C
S3150800BDF01188BFF36F8FBFF34F8FFEE7013B0365D3
S3150800BE00C16AC26C91421DD00BB1002038BD051D18
S3150800BE102846FEF7C5FCE06CE062C0F13803A36172
S3150800BE200A4B1B68984201D9084B186000EB800042
S3150800BE302946074B03EB8000FEF78EFC0120E5E759
S3150800BE40002070470020E1E774110020980C0020BC
S3150800BE50140D0020002846D038B50446036D43B9B2
S3150800BE604FF0500383F31188BFF36F8FBFF34F8FE3
S3150800BE70FEE7C26C8A4200D20A46E16A914201D0C4
S3150800BE80012B00D038BD184B1B68A34222D0E262B2
S3150800BE90A369002B02DBC2F13802A261626901EBD9
S3150800BEA08101124B03EB81039A42EBD1251D2846EB
S3150800BEB0FEF776FCE06A0E4B1B68984201D90C4BDC
S3150800BEC0186000EB80002946084B03EB8000FEF75C
S3150800BED043FCD7E74FF0500383F31188BFF36F8F06
S3150800BEE0BFF34F8FFEE7704774110020140D002032
S3150800BEF0980C0020044A136898691368DB6A12686C
S3150800BF00C3F138039361704774110020054B1B6811
S3150800BF1023B1044B1A68136D01331365014B186876
S3150800BF20704700BF74110020064B1A6813682BB9B6
S3150800BF300123036023B9D368186870470023F8E71C
S3150800BF40002070477812002008B5416000619142D0
S3150800BF500CD8D21A83699A4201D3012008BD011D63
S3150800BF60094B1868FEF703FC0020F7E79A4201D24E
S3150800BF70994206D2011D054B1868FEF7F8FB00200A
S3150800BF80ECE70120EAE700BF7412002078120020CF
S3150800BF9030B583B000F0EEFA114B1B681BB100F008
S3150800BFA00BFB03B030BD0F4D2846FEF7C7FB0E4C02
S3150800BFB02046FEF7C3FB0D4B1D600D4B1C6000238E
S3150800BFC000930C4B0C4A10210A20FEF7F7FC044B91
S3150800BFD018600028E3D00949FFF7C8F8DFE700BF73
S3150800BFE070120020901200207C1200207812002087
S3150800BFF07412002078110020C81100200CCE000809
S3150800C0002DE9F041079F41B94FF0500383F311889A
S3150800C010BFF36F8FBFF34F8FFEE7064614461D46E4
S3150800C02088468FB1FFF7B4FF3E60C7F81880FD61F8
S3150800C030069B3B62381DFEF78CFB2CB197F828301F
S3150800C04043F0040387F82830BDE8F08110B588B0BE
S3150800C050FFF79EFF124B1B68CBB10024059406948C
S3150800C06007AA06A905A8FEF703FA059B0293069BED
S3150800C0700193022300932346079A0A490A48FFF7C1
S3150800C0804DFA0A4B186010B1012008B010BD4FF0E8
S3150800C090500383F31188BFF36F8FBFF34F8FFEE70B
S3150800C0A07012002014CE00083DC400086C1200204F
S3150800C0B02DE9F04182B00446884617461D462C20D5
S3150800C0C000F010FC064658B1002380F8283001908D
S3150800C0D0089B00932B463A4641462046FFF790FFB9
S3150800C0E0304602B0BDE8F08110B584B084462C20F5
S3150800C0F0039003982C2808D04FF0500383F3118837
S3150800C100BFF36F8FBFF34F8FFEE70398079860B1B1
S3150800C1100220079C84F8280001940698009060463F
S3150800C120FFF76EFF079804B010BD4FF0500383F376
S3150800C1301188BFF36F8FBFF34F8FFEE7B8B19C46E8
S3150800C14003461848006858B300B585B000910192B7
S3150800C150029305291CDCFFF7D9FD022810D000231D
S3150800C1601A4669460F480068FEF796FC15E04FF038
S3150800C170500383F31188BFF36F8FBFF34F8FFEE72A
S3150800C1800023069A694607480068FEF785FC04E01E
S3150800C190002362466946FEF789FD05B05DF804FB93
S3150800C1A0002070477012002070B582B01B4B1B68C8
S3150800C1B01A6862B3DB681E68DC68251D2846FEF728
S3150800C1C0EFFA236A2046984794F8283013F0040FAC
S3150800C1D0ECD0A36933449E4207D2636024612946A2
S3150800C1E00E4B1868FEF7C3FAE0E7002100910B46EC
S3150800C1F032462046FFF7A2FF0028D7D14FF050035A
S3150800C20083F31188BFF36F8FBFF34F8FFEE7044A9E
S3150800C210106802490860136002B070BD78120020E9
S3150800C2207412002038B50546FFF744FA0446074B52
S3150800C2301B68834205D800232B60044B1C602046EC
S3150800C24038BDFFF7B1FF01232B60F6E7681200201F
S3150800C25070B582B006460D4617490968C968CC68A4
S3150800C260201DFEF79DFA94F828C01CF0040F08D18B
S3150800C2702CF0010C84F828C0236A2046984702B09F
S3150800C28070BDA16933462A4631442046FFF75CFE55
S3150800C2900028F1D0002100910B4632462046FFF7D0
S3150800C2A04DFF0028E8D14FF0500383F31188BFF300
S3150800C2B06F8FBFF34F8FFEE77812002070B582B0FC
S3150800C2C006460C46FFF7EEF901A8FFF7ABFF019B00
S3150800C2D033BB0546E4B9B04213D22246711B124B52
S3150800C2E01868FEF757FFFFF777FAD8B94FF0E0233B
S3150800C2F04FF08052C3F8042DBFF34F8FBFF36F8FF3
S3150800C30010E0FFF769FA29463046FFF7A1FF09E072
S3150800C310064A126812680AB90124DEE71C46DCE7F9
S3150800C320FFF75AFA02B070BD70120020741200208E
S3150800C33010B588B002E0049B002B0FDA002204A98E
S3150800C3403D4B1868FEF719FD002873D0049B002B97
S3150800C350F1DA07990698059B9847ECE7069C636906
S3150800C36013B1201DFEF71CFA03A8FFF75BFF049B19
S3150800C370092BE3D8DFE803F0050505303750050536
S3150800C380303794F8283043F0010384F82830059BA9
S3150800C390A169024619442046FFF7D6FD0028CDD0EC
S3150800C3A0236A2046984794F8283013F0040FC5D01E
S3150800C3B0A269002100910B46059802442046FFF722
S3150800C3C0BDFE0028BAD14FF0500383F31188BFF39E
S3150800C3D06F8FBFF34F8FFEE794F8283023F00103E1
S3150800C3E084F82830AAE794F8283043F0010384F843
S3150800C3F028300599A16131B1034602460144204619
S3150800C400FFF7A2FD9AE74FF0500383F31188BFF3B5
S3150800C4106F8FBFF34F8FFEE794F8283013F0020FA3
S3150800C42004D023F0010384F8283087E7204600F07B
S3150800C430DBFA83E708B010BD7012002000B583B0A0
S3150800C44001A8FFF771FD0199FFF738FFFFF770FFA5
S3150800C450F6E740B110B5044600F08CF8E46900F040
S3150800C460ABF8204610BD4FF0500383F31188BFF395
S3150800C4706F8FBFF34F8FFEE710B584B014461A4688
S3150800C4806FF001030093019002910394002369461B
S3150800C49002480068FEF70AFC04B010BD70120020BE
S3150800C4A082B0002301930D4B1B68B3F1FF3F08D000
S3150800C4B04FF0500383F31188BFF36F8FBFF34F8F8D
S3150800C4C0FEE74FF0500383F31188BFF36F8FBFF376
S3150800C4D04F8F019B002BFCD002B07047C400002090
S3150800C4E008480068006880F308884FF0000080F369
S3150800C4F0148862B661B6BFF34F8FBFF36F8F00DF44
S3150800C50000BF000008ED00E0DFF80C00016841F408
S3150800C510700101607047000088ED00E04FF08073FD
S3150800C52040F8043C21F0010140F8081C054B40F88E
S3150800C5300C3C40F8202C6FF0020340F8243C4438A9
S3150800C540704700BFA1C400080000000000000000FA
S3150800C550074B19680868B0E8F04F80F30988BFF3FD
S3150800C5606F8F4FF0000080F311887047AFF300809B
S3150800C570741100204FF0500383F31188BFF36F8FB7
S3150800C580BFF34F8F0B4A136801331360012B00D09A
S3150800C59070474FF0E023D3F8043D13F0FF0FF7D0B0
S3150800C5A04FF0500383F31188BFF36F8FBFF34F8F9C
S3150800C5B0FEE700BFC4000020094B1B6843B94FF0D3
S3150800C5C0500383F31188BFF36F8FBFF34F8FFEE7D6
S3150800C5D0013B034A13600BB983F31188704700BF08
S3150800C5E0C400002000000000000000000000000059
S3150800C5F0EFF30980BFF36F8F154B1A681EF0100F03
S3150800C60008BF20ED108A20E9F04F10602DE90900D7
S3150800C6104FF0500080F31188BFF34F8FBFF36F8F31
S3150800C620FFF77CF94FF0000080F3118809BC196800
S3150800C6300868B0E8F04F1EF0100F08BFB0EC108A7B
S3150800C64080F30988BFF36F8F704700BFAFF3008090
S3150800C6507411002008B54FF0500383F31188BFF317
S3150800C6606F8FBFF34F8FFFF72BF828B14FF0E023FA
S3150800C6704FF08052C3F8042D002383F3118808BDB8
S3150800C6804FF0E022002313619361054B1B680549AF
S3150800C690A1FB03139B09013B5361072313617047F1
S3150800C6A094000020D34D62104FF0E023D3F8002DFC
S3150800C6B03D4B9A421CD04FF0E023D3F8002D3B4B5C
S3150800C6C09A421ED030B583B0394B1A78D2B201924D
S3150800C6D0FF221A701B78DBB28DF803309DF8033001
S3150800C6E003F05003334A1370334B07221A601BE0DA
S3150800C6F04FF0500383F31188BFF36F8FBFF34F8F4B
S3150800C700FEE74FF0500383F31188BFF36F8FBFF333
S3150800C7104F8FFEE7284A1368013B13609DF80330E4
S3150800C7205B00DBB28DF803309DF8033013F0800F01
S3150800C730F0D1214B1B68032B08D04FF0500383F32D
S3150800C7401188BFF36F8FBFF34F8FFEE71B021A4A9C
S3150800C750136003F4E0631360019BDBB2144A1370A1
S3150800C7604FF0E024D4F8203D43F47003C4F8203D8C
S3150800C770D4F8203D43F07043C4F8203DFFF780FF0E
S3150800C78000250E4B1D60FFF7BFFED4F8343F43F07B
S3150800C7904043C4F8343FFFF7A3FEFFF7BFF8FFF79F
S3150800C7A07FFE284603B030BD71C20F4170C20F41EB
S3150800C7B000E400E0A8120020A4120020C400002013
S3150800C7C0EFF305830F2B0FD9114A9B5CDBB2114A95
S3150800C7D012789A4208D94FF0500383F31188BFF3B1
S3150800C7E06F8FBFF34F8FFEE74FF0E023D3F80C3D72
S3150800C7F003F4E063084A1268934208D94FF05003DD
S3150800C80083F31188BFF36F8FBFF34F8FFEE770472F
S3150800C810F0E300E0A8120020A4120020124A12F049
S3150800C820070F1ED0D11D21F00701C1F5004313449F
S3150800C8300A460E480260002141601344083B23F073
S3150800C84007030B48036059601960991A5160136011
S3150800C850084B1960084B1960084B4FF000421A60E4
S3150800C86070474FF40043E4E7CC120020C4120020BE
S3150800C870C0120020B8120020BC120020AC12002002
S3150800C880164B1A461B688342FBD3516802EB010C10
S3150800C890844509D0416800EB010C634509D0036063
S3150800C8A0904219D0106070474068014451601046A4
S3150800C8B0F0E710B40A4C2468A3420BD05B6819440D
S3150800C8C0416013681B680360904200D010605DF8F1
S3150800C8D0044B70470460F7E7704700BFC412002096
S3150800C8E0C012002038B50446FEF7DCFE384B1B683C
S3150800C8F0B3B1384B1B681C4250D1002C50D004F100
S3150800C900080214F0070F02D022F007020832002AA4
S3150800C91055D0314B1B68934253D330490C6804E019
S3150800C920FFF77CFFE5E721461C466368934202D27F
S3150800C9302368002BF7D1264B1B68A34243D00D680A
S3150800C940083523680B6063689B1A102B10D9A0184A
S3150800C95010F0070F08D04FF0500383F31188BFF388
S3150800C9606F8FBFF34F8FFEE743606260FFF788FF64
S3150800C970626819490B689B1A0B60194909688B424A
S3150800C98001D217490B60134B1B68134363600023DE
S3150800C9902360144A13680133136002E0002500E09F
S3150800C9A00025FEF719FF15F0070F0ED04FF05003BC
S3150800C9B083F31188BFF36F8FBFF34F8FFEE7002510
S3150800C9C0EFE70025EDE70025EBE7284638BD00BF71
S3150800C9D0C0120020AC120020BC120020C412002095
S3150800C9E0B8120020B4120020002834D038B5044606
S3150800C9F0A0F1080550F8043C174A1268134208D1FA
S3150800CA004FF0500383F31188BFF36F8FBFF34F8F37
S3150800CA10FEE750F8081C41B14FF0500383F3118824
S3150800CA20BFF36F8FBFF34F8FFEE723EA020340F889
S3150800CA30043CFEF737FE54F8041C084A13680B44F6
S3150800CA4013602846FFF71CFF054A13680133136075
S3150800CA50FEF7C2FE38BD7047AC120020BC1200209B
S3150800CA60B0120020DFF834D0F8F7A4FC0C480D49C2
S3150800CA700D4A002302E0D458C4500433C4188C422B
S3150800CA80F9D30A4A0A4C002301E013600432A24291
S3150800CA90FBD300F077F8F8F7F9F9FEE700C00020B5
S3150800CAA000000020180100200CD3000818010020FF
S3150800CAB00C940020FEE702440346934200D17047D7
S3150800CAC003F8011BF9E700002D4B1B68834270B57C
S3150800CAD0044653D0C3691BB3DB6863B10025E36919
S3150800CAE0DB685959B1B90435802DF8D1E369204678
S3150800CAF0D96800F07BF8E369196811B1204600F09F
S3150800CB0075F8E3699D685DB1294620462D6800F0F1
S3150800CB106DF8F8E70E68204600F068F83146E1E758
S3150800CB20616911B1204600F061F8E16911B120464A
S3150800CB3000F05CF8216B11B1204600F057F8616BE4
S3150800CB4011B1204600F052F8A16B11B1204600F051
S3150800CB504DF8A16C11B1204600F048F8616C11B18E
S3150800CB60204600F043F8E16A11B1204600F03EF88D
S3150800CB70236A1BB12046BDE87040184770BD00BF48
S3150800CB80C800002070B50D4D0D4C641BA41000267E
S3150800CB90A64209D10B4D0C4C00F07EF8641BA4107C
S3150800CBA00026A64205D170BD55F8043B98470136C4
S3150800CBB0EEE755F8043B98470136F2E704D3000838
S3150800CBC004D3000804D3000808D300087047704748
S3150800CBD00A44914200F1FF3300D1704710B511F8AD
S3150800CBE0014B03F8014F9142F9D110BD38B50546FE
S3150800CBF0002941D051F8043C0C1F002BB8BFE4189B
S3150800CC0000F03EF81D4A136833B96360146028467D
S3150800CC10BDE8384000F03AB8A34208D92068211880
S3150800CC208B4201BF19685B6809182160EDE71A464F
S3150800CC305B680BB1A342FAD911685018A0420BD110
S3150800CC4020680144501883421160E0D118685B6877
S3150800CC50536008441060DAE702D90C232B60D6E744
S3150800CC60206821188B4204BF19685B68636004BF9B
S3150800CC70091821605460CAE738BD00BF089400202F
S3150800CC800148FFF7A3BF00BF049400200148FFF73F
S3150800CC909EBF00BF04940020F8B500BFF8BC08BCCE
S3150800CCA09E467047F8B500BFF8BC08BC9E4670475C
S3150800CCB0494E49545F546872656164004D41494E56
S3150800CCC05F5761746368646F670000004D41494EA1
S3150800CCD05F55706461746554696D65720000000083
S3150800CCE04D41494E5F4576656E745F466C61677364
S3150800CCF0000000004D41494E5F43414E5F52785F48
S3150800CD0051756575650000004D41494E5F5468725E
S3150800CD10656164005045434F5F4576656E745F46AE
S3150800CD206C616773000000005045434F5F5570649F
S3150800CD3061746554696D6572000000005045434F83
S3150800CD405F54687265616400564152485F4D757458
S3150800CD5065780000414443445F4D7574657800006A
S3150800CD60414E50495F4D757465780000414E5049F3
S3150800CD705F4576656E745F466C61677300000000F8
S3150800CD80414E50495F54687265616400414E504F88
S3150800CD905F4576656E745F466C61677300000000D8
S3150800CDA0414E504F5F55706461746554696D657284
S3150800CDB000000000414E504F5F5468726561640080
S3150800CDC0535049445F4576656E745F466C61677378
S3150800CDD000000000535049445F4144435F4D757459
S3150800CDE06578000054454D505F546872656164006B
S3150800CDF05553464C5F4D7574657800004465666109
S3150800CE00756C740049444C4500000000546D72511D
S3150800CE1000000000546D722053766300B0CC000801
S3150800CE2000000000000000000000000000000000F4
S3150800CE30000400002F0000000000000000000000B1
S3150800CE40BCCC000800000000000000000000000044
S3150800CE50CCCC000800000000000000000000000024
S3150800CE60E0CC000800000000000000000000000000
S3150800CE70F4CC0008000000000000000000000000DC
S3150800CE80000000000000000008CD000800000000B7
S3150800CE900000000000000000000000000004000080
S3150800CEA021000000000000000000000014CD00086A
S3150800CEB000000000000000000000000028CD000867
S3150800CEC00000000000000000000000003CCD000843
S3150800CED00000000000000000000000000000000044
S3150800CEE00004000028000000000000000000000008
S3150800CEF048CD000803000000000000000000000004
S3150800CF000000000001000000000000000100000011
S3150800CF1001000000000000000000A0C00000404121
S3150800CF201100000000000000000000000000C842D8
S3150800CF301100000000000000000000000000C842C8
S3150800CF401100000000000000000000000000C842B8
S3150800CF50010000000000B841000020C2000048425D
S3150800CF6011000000000020410000000000004041C0
S3150800CF7011000000000000C00000A0C00000000072
S3150800CF800900000000000000000048C200004842F6
S3150800CF900900000000000000000048C200004842E6
S3150800CFA0090000000000000000007AC400007A446E
S3150800CFB00900000000000000000000C100007041E8
S3150800CFC00900000000000000000020C10000204108
S3150800CFD009000000000000000000000000002041D9
S3150800CFE00900000000000000000048C200001643C7
S3150800CFF009000000000000000000A0410000F04108
S3150800D0000900000000000000000020C10000C04028
S3150800D0100900000000000000000020C100001643BF
S3150800D02008000000000000000000000001000000E9
S3150800D030080000000000000000000000FFFFFFFFDE
S3150800D0401100000033335340020000000000804006
S3150800D05054CD000803000000000000000000000096
S3150800D06060CD00080300000000000000000000007A
S3150800D0706CCD000800000000000000000000000061
S3150800D08080CD00080000000000000000000000003D
S3150800D090000000000004000010000000000000006E
S3150800D0A00000000000000000000000000100000071
S3150800D0B00100000000000000000004419A996D413B
S3150800D0C000000441000020410000A040000020416B
S3150800D0D00000A0408CCD0008000000000000000001
S3150800D0E000000000A0CD00080000000000000000BD
S3150800D0F000000000B4CD0008000000000000000099
S3150800D10000000000000000000004000018000000F5
S3150800D1100000000000000000000400484000000075
S3150800D12001000000000000000100000000000000EF
S3150800D1300100000000000000000400482000000074
S3150800D14001000000000000000100000000000000CF
S3150800D1500100000000000000000800480040000030
S3150800D16001000000000000000100000000000000AF
S3150800D1700000000001000000000000480001000057
S3150800D180010000000000000001000000000000008F
S3150800D19000000000010000000004004880000000B4
S3150800D1A00000000000000000010000000000000070
S3150800D1B00000000001000000000800480080000090
S3150800D1C00000000000000000010000000000000050
S3150800D1D000000000010000000004004808000000EC
S3150800D1E00000000000000000010000000000000030
S3150800D1F000000000010000000004004810000000C4
S3150800D200000000000000000001000000000000000F
S3150800D2100000000001000000000000480080000037
S3150800D22000000000000000000100000000000000EF
S3150800D23000000000010000000003002000000000BC
S3150800D2405CD200080100000002000000C0CD000802
S3150800D250000000000000000000000000D4CD000817
S3150800D260030000000000000000000000E4CD0008F4
S3150800D27000000000000000000000000000000000A0
S3150800D2800004000018000000000000000000000074
S3150800D290F0CD0008030000000000000000000000B8
S3150800D2A0FCCD00080000000000000000000000009F
S3150800D2B00000000000020000180000000000000046
S3150800D2C000000000A0860100400D0300801A060039
S3150800D2D000350C0040420F0080841E0000093D0006
S3150800D2E000127A000024F40000366E010048E801B6
S3150800D2F0006CDC02000000000000000001020304CC
S3090800D30006070809FD
S3090800D304B529000831
S3090800D3089129000851
S3150800D30C00FF0000080200201002002000000000A8
S3150800D31C00000000000000000000000000000000F3
S3150800D32C00000000000000000000000000000000E3
S3150800D33C00000000000000000000000000000000D3
S3150800D34C000000000060000000000000E0E900009A
S3150800D35C00000000000000000100000000000000B2
S3150800D36C0100000001000000000000000040000061
S3150800D37C0000000000E800000000000000000000AB
S3150800D38C0000000000000000010000000100000081
S3150800D39C0000000000093D0001000000100000001C
S3150800D3AC0000000000000000000000000000000063
S3150800D3BC0100000000000000000000000000000052
S3150800D3CC20000000AAAAAAAACC000020000000008F
S3150800D3DCCC920020349300209C930020000000007F
S3150800D3EC0000000000000000000000000000000023
S3150800D3FC0000000000000000000000000000000013
S3150800D40C0000000000000000000000000000000002
S30D0800D41C0000000000000000FA
S7050800CA65C3
